:020000040800F2
:1000000090320020713D000861040008630400087C
:10001000670400086B0400086F040008000000007B
:100020000000000000000000000000007304000851
:100030007504000800000000770400087904000837
:100040008B3D00088B3D00088B3D00088B3D000870
:100050008B3D00088B3D00088B3D00088B3D000860
:100060008B3D00088B3D00088B3D00088B3D000850
:100070008B3D00088B3D00088B3D00088B3D000840
:100080008B3D00088B3D00088B3D00088B3D000830
:100090008B3D00088B3D00088B3D00088B3D000820
:1000A0008B3D00088B3D00088B3D00088B3D000810
:1000B0008B3D00088B3D0008B90200088B3D00080D
:1000C0008B3D00088B3D00088B3D00088B3D0008F0
:1000D0008B3D0008FD3C0008AB3B0008633C00087A
:1000E0008B3D00088B3D00088B3D00088B3D0008D0
:1000F0008B3D00088B3D00088B3D00088B3D0008C0
:100100008B3D00088B3D00088B3D00088B3D0008AF
:100110008B3D00088B3D00088B3D00088B3D00089F
:100120008B3D00088B3D00088B3D00088B3D00088F
:1001300000F002F800F0B0F80AA090E8000C824449
:100140008344AAF10107DA4501D100F0A5F8AFF226
:10015000090EBAE80F0013F0010F18BFFB1A43F0A5
:10016000010318475CA800007CA800000A444FF077
:10017000000C10F8013B13F0070408BF10F8014B06
:100180001D1108BF10F8015B641E05D010F8016B4B
:10019000641E01F8016BF9D113F0080F1EBF10F8AF
:1001A000014BAD1C0C1B09D16D1E58BF01F801CBD2
:1001B000FAD505E014F8016B01F8016B6D1EF9D555
:1001C0009142D6D37047000000230024002500266A
:1001D000103A28BF78C1FBD8520728BF30C148BFAA
:1001E0000B6070476E2905F05187702905F0ED848A
:1001F000662907F02381652907F02081672907F028
:100200001D816129AFF3008003681B0A28BF41F0FC
:100210008001692905F0FE86642905F0FB867529B1
:1002200005F0F8866F2906F04880782905F0B98432
:10023000E92905F0E387E42905F0E087F52905F0D1
:10024000DD87EF2906F04580F82905F0B8840368BA
:10025000DB0928BF41F08001632905F0528773292B
:1002600005F05787E32906F04683F32906F04B8310
:10027000002070471FB506F0CDFB040000200021D0
:1002800007F0C6F8401C60600020002107F0AAF8C3
:10029000E0601FBD10B510BD06F08FFB1146FFF7E3
:1002A000E9FF00F049F806F06BFC03B4FFF7F2FF3A
:1002B00003BC03F013FB000010B501214D4805F00D
:1002C000DCFB4D4908700846007818B10121494807
:1002D00005F0DCFB10BD1FB50121042004F0FFF880
:1002E00044F61F60ADF808004720ADF80400002078
:1002F000ADF80A00ADF806003E4804F0D1FC01A9B3
:100300003C4804F0A1FD01213A4805F0F9F801222A
:100310001146384805F00FF91E208DF80000022024
:100320008DF8010000208DF8020001208DF80300F7
:10033000684603F042FD1FBD1CB54FF4A06003F0FA
:1003400037FD03F061FA02F0F1FF4FF4E13003F002
:10035000D4FA4FF4E13003F022FB4FF47A7003F04B
:1003600090FA26A005F0BCFB00F0DAFB00F06DFA75
:10037000FFF7B1FF03F0B4F80AE0322003F081FA8E
:100380002048006808B9012000E000201D490860ED
:1003900003F086F84EF617718842EED10C201AA1B0
:1003A0000346C822CDE900100021084601F002F8FA
:1003B0000C201BA103466422CDE900100F21002070
:1003C00000F0F8FF0C201AA103466422CDE90010CA
:1003D0001E21002000F0EEFF00F0C1FE40F2DC50D4
:1003E00003F04FFA0022022115A000F038FD00BFF3
:1003F000FEE700000008004000000020696E6974FC
:100400000D0A000094012342BAFEC4CFB9A4D2B5AC
:10041000D6B0D2B5BCBCCAF5D1A7D4BA0000000092
:10042000C1F5BAC67361646C666A617366000000E8
:100430007361646C666A6173666A6C616B0000006C
:1004400071725F74657374B5A5C6ACBBFAC9FAB3B3
:10045000C9B6FECEACC2EB313233343536000000C3
:10046000704700BFFEE700BFFEE700BFFEE700BF2A
:10047000FEE7704770477047704700000CB50020DA
:10048000019000906C48006840F480306A49086030
:1004900000BF6948006800F4003000900198401CDB
:1004A0000190009818B90198B0F5A06FF1D1624899
:1004B000006800F4003010B10120009001E000203D
:1004C00000900098012843D15C48006840F010007B
:1004D0005A4908600846006820F003000860084692
:1004E000006840F002000860534840685249486084
:1004F0000846406848600846406840F480604860AC
:100500000846406820F47C1048600846406840F483
:10051000E81048600846006840F08070086000BF3E
:100520004548006800F000700028F9D04248406853
:1005300020F00300404948600846406840F002004F
:10054000486000BF3C48406800F00C000828F9D122
:100550000CBD10B5FFF792FF10BD10B5364800680E
:1005600040F00100344908600846406834490840BA
:100570003149486008460068324908402E49086001
:100580000846006820F4802008600846406820F48F
:10059000FE0048604FF41F008860FFF7DAFF4FF05D
:1005A00000602949086010BD10B50021002000221C
:1005B000214B5B6803F00C0121B1042906D0082906
:1005C00028D107E0214B224C236027E01F4B204C11
:1005D000236023E0184B5B6803F47010164B5B68D4
:1005E00003F48032022303EB904022B9194B4343BA
:1005F000174C23600DE0104B5B6803F4003323B10C
:10060000144B4343124C236003E0104B4343104C04
:10061000236003E00D4B0E4C236000BF00BF064B70
:100620005B68C3F303130C4CE15C094B1B68CB40C4
:10063000074C236010BD0000001002400020024063
:100640000000FFF8FFFFF6FE08ED00E000127A0060
:100650000400002000093D000800002010B504211E
:10066000FB4803F020FD4FF48061FA4803F01BFDC6
:100670004FF48061F74803F018FD0421F44803F0BB
:1006800014FD10BD10B50421F14803F00CFD4FF42A
:100690008061F04803F009FD4FF48061ED4803F0FC
:1006A00002FD10BD10B50421E94803F0FCFC042153
:1006B000E74803F0FAFC10BD2DE9F04105462C4651
:1006C0000421E34803F0F1FC00261AE0274607F076
:1006D0008007802F04D1F900DE4803F0E4FC04E039
:1006E0004FF48061DB4803F0E0FC6006040E042157
:1006F000D74803F0D8FC0421D54803F0D6FC701C81
:10070000C6B2082EE2DBBDE8F08110B50446FFF763
:10071000A5FF7820FFF7D0FFFFF7C4FF0020FFF709
:10072000CBFFFFF7BFFF2046FFF7C6FFFFF7BAFF7B
:10073000FFF7A8FF10BD10B50446FFF78FFF782024
:10074000FFF7BAFFFFF7AEFF4020FFF7B5FFFFF757
:10075000A9FF2046FFF7B0FFFFF7A4FFFFF792FFC6
:1007600010BD70B504460D461DB1E0B2FFF7E3FFC2
:1007700002E0E0B2FFF7C9FF70BD70B50646002485
:1007800018E004F1B0000021FFF7EBFF002108465C
:10079000FFF7E7FF00211020FFF7E3FF002505E04A
:1007A00001213046FFF7DDFF681CC5B2802DF7DB65
:1007B000601CC4B2082CE4DB70BD06E041F66501A4
:1007C00000E0491E0029FCD1401E0028F6D17047E8
:1007D000014605E0002001E0421CD0B27B28FBDB93
:1007E0000A1EA1F10101F5D1704770B504460D460E
:1007F00005F1B0000021FFF7B4FF102141EA141009
:100800000021FFF7AEFF04F00F000021FFF7A9FF62
:1008100070BD10B500218D20FFF7A3FF002114202B
:10082000FFF79FFF0021AF20FFF79BFF10BD10B522
:1008300000218D20FFF795FF00211020FFF791FF89
:100840000021AE20FFF78DFF10BD70B5002418E029
:1008500004F1B0000021FFF784FF00210846FFF7F4
:1008600080FF00211020FFF77CFF002505E001211B
:100870000020FFF776FF681CC5B2802DF7DB601CF7
:10088000C4B2082CE4DB70BD70B5002418E004F19C
:10089000B0000021FFF765FF00210846FFF761FF68
:1008A00000211020FFF75DFF002505E0012108462B
:1008B000FFF757FF681CC5B2802DF7DB601CC4B280
:1008C000082CE4DB70BD2DE9F04707460E46904644
:1008D000994600250024A8F12000C5B27F2F02DD33
:1008E0000027B01CC6B2B9F1100F24D131463846EA
:1008F000FFF77BFF002408E004EB0511564A505C2B
:100900000121FFF72EFF601CC4B2082CF4DB701C21
:10091000C1B23846FFF769FF002409E004EB051176
:1009200008314D4A505C0121FFF71BFF601CC4B227
:10093000082CF3DB12E031463846FFF756FF00245F
:100940000AE005EB4501454A02EB4101085D012142
:10095000FFF707FF601CC4B2062CF2DBBDE8F0878E
:1009600010B50246012000E050430B1EA1F1010426
:10097000E1B2F9D110BD2DE9FF5F074691461E4651
:100980000E9D4FF0000A002435E0301B401EC1B21E
:100990000A20FFF7E5FFB9FBF0F00A21B0FBF1F206
:1009A00001FB1208BAF1000F14D1701EA04211DD34
:1009B000B8F1000F0CD1AB4605EBDB71491001FB20
:1009C0000471C8B22B4620220199FFF77CFF10E08A
:1009D0004FF0010AAB4605EBDB71491001FB0471D6
:1009E000C8B208F13001CAB22B460199FFF76BFF7C
:1009F00000BF601CC4B2B442C7DBBDE8FF9F2DE955
:100A0000F04104460F461546984600260FE0AA5DC1
:100A1000434639462046FFF756FF04F10800C4B2AA
:100A2000782C02DD0024B81CC7B2701CC6B2A85DC9
:100A30000028ECD1BDE8F0812DE9F04180460E465A
:100A40001546002731464046FFF7CFFE002412E04E
:100A5000000C0140001C014068760008407400084A
:100A6000F74A02EB8511085D0121FFF77AFE781C39
:100A7000C7B2601CC4B2102CF2DB701CC1B240467D
:100A8000FFF7B3FE00240CE06900491CEC4A02EBBE
:100A90004111085D0121FFF764FE781CC7B2601C9C
:100AA000C4B2102CF0DBBDE8F0812DE9F05F064602
:100AB0000F4690461C46DDF828A04FF0000BE117CA
:100AC00004EB5171C910A4EBC10131B92046E11703
:100AD00004EB5171C1F3C70506E02046E11704EBB2
:100AE0005171C910491CCDB23D4615E0294630462A
:100AF000FFF77BFEB1460BE059460BF1010B1AF8EC
:100B000001000121FFF72DFE09F1010000F0FF09AE
:100B1000C145F1DB681CC5B2A542E7DBBDE8F09F2B
:100B200008B50121082003F0CDFC0420ADF8000039
:100B300010208DF8030003208DF802006946C1489B
:100B400003F004FA0421BF4803F0ADFA012180202C
:100B500003F0B8FC4FF48060ADF8000010208DF871
:100B6000030003208DF802006946B74803F0EEF950
:100B70004FF48061B44803F096FA4FF4487002F0E5
:100B800080FE0021AE20FFF7ECFD0021D520FFF70D
:100B9000E8FD00215020FFF7E4FD0021A820FFF729
:100BA000E0FD00213F20FFF7DCFD0021D320FFF70F
:100BB000D8FD00210846FFF7D4FD00214020FFF7B3
:100BC000D0FD00218D20FFF7CCFD00211420FFF780
:100BD000C8FD00212020FFF7C4FD00210220FFF7FF
:100BE000C0FD0021A120FFF7BCFD0021C020FFF7C0
:100BF000B8FD0021DA20FFF7B4FD00211220FFF735
:100C0000B0FD00218120FFF7ACFD0021EF20FFF7B0
:100C1000A8FD0021D920FFF7A4FD0021F120FFF756
:100C2000A0FD0021DB20FFF79CFD00213020FFF715
:100C300098FD0021A420FFF794FD0021A620FFF7D6
:100C400090FD0021AF20FFF78CFD08BD70B500249A
:100C50001BE004F1B0000021FFF783FD00210846EE
:100C6000FFF77FFD00211020FFF77BFD002508E046
:100C7000764901EBC501085D0121FFF772FD681C93
:100C8000C5B2802DF4DB601CC4B2082CE1DB70BD62
:100C900070B500240CE0002506E000206B4901EB54
:100CA000C5010855681CC5B2802DF6DB601CC4B2B6
:100CB000082CF0DBFFF7CAFF70BDF0B51446002624
:100CC0007F2801DC3F2900DDF0BD0B46CF1701EB8B
:100CD0005777FF10C7F10707FAB2CF1701EB577725
:100CE000FF10A1EBC707FDB2C5F107070123BB4009
:100CF000DEB24CB1554B03EBC0039B5C3343534F07
:100D000007EBC007BB5408E0504B03EBC0039B5CF0
:100D1000B3434E4F07EBC007BB5400BFD4E72DE9E8
:100D2000F04704468A4615469946AC4202DD2F46F6
:100D3000A04601E02746A8463E4606E04A46514600
:100D40003046FFF7BAFF701CC6B24645F6DDFFF726
:100D50007DFFBDE8F0872DE9F04782460C46154639
:100D60009946AC4202DD2F46A04601E02746A84640
:100D70003E4606E04A4631465046FFF79EFF701C4D
:100D8000C6B24645F6DDFFF761FFBDE8F0872DE905
:100D9000F84F0746884615461E46B04502DDB14667
:100DA000C24601E0C146B246AF4202DDAB46009703
:100DB00001E0BB4600955C460BE0414620460A9A9E
:100DC000FFF77BFF314620460A9AFFF776FF601C4B
:100DD000C4B200988442F0DD4C460BE02146384610
:100DE0000A9AFFF76AFF214628460A9AFFF765FF2D
:100DF000601CC4B25445F1DDFFF728FFBDE8F88F51
:100E00002DE9F04706460F4690469946DDF820A0AA
:100E100034460CE03D4606E0524629462046FFF7A0
:100E20004CFF681CC5B24D45F6DB601CC4B244459E
:100E3000F0DBBDE8F08710B50246012009E00000B4
:100E4000587C0008000C0140001C01408801002073
:100E500050430B1EA1F10104E1B2F9D110BD2DE9FF
:100E6000F74F82B08A4693460124BBF1000F01D0B0
:100E7000A04601E04FF00008029801F071FFFD4824
:100E80000068402191FBF0F0C4B2FA49096861435F
:100E9000C1F1400000EBD071C1F3470505EB0A003A
:100EA000C6B2B8F1000F15D101200090F1480068DA
:100EB00004FB0050801CC3B2EE48006804FB0060D5
:100EC000801CC2B2A81EC1B2B01E00F0FF0C60466A
:100ED000FFF796FF00273CE04FF000092DE007EBFD
:100EE0004700C0EB8710E449084410F809000128C6
:100EF0000AD108F0FF0000902819C3B23019C2B21D
:100F000029463046FFF77CFF07EB4700C0EB871010
:100F1000D949084410F8090058B9C8F10100C0B215
:100F200000902819C3B23019C2B229463046FFF7E3
:100F300067FF2819C5B209F10109CE48006881454B
:100F4000CDD33019C6B2CB48006800FB1450C5B2EF
:100F50007F1CC84800688742BED3FFF777FE05B004
:100F6000BDE8F08F0FB430B585B004460D460020C3
:100F700001900290039004900BA8009001A8009AA1
:100F80000A9904F09BFD00200090102301AA294635
:100F90002046FFF734FD05B030BC5DF814FBF0B51A
:100FA000144600267F2801DC3F2900DDF0BD0B46FA
:100FB000CF1701EB5777FF10C7F10707FAB2CF172A
:100FC00001EB5777FF10A1EBC707FDB2C5F107078B
:100FD0000123BB40DEB24CB1A84B03EBC0039B5CCA
:100FE0003343A64F07EBC007BB5408E0A34B03EB0A
:100FF000C0039B5CB343A14F07EBC007BB5400BFCA
:10100000D4E72DE9F84F80460F4616461C46BA46EF
:101010002046E31704EB5373DB1021464FEAE47CD0
:1010200004EB5C7C4FEAEC0CA4EBCC0CBCF1000FA5
:1010300002D04FF0010C01E04FF0000C6344224657
:1010400004EBD27C4FEA6C0C03FB0CF303F0FF0BB8
:10105000A6F12000C6B200254EE00C2C07D106EB0D
:101060004600874901EB8000405D009013E0102CA2
:1010700005D1844800EB0610405D00900BE0182C71
:1010800007D106EBC600804901EB8000405D00906F
:1010900001E0BDE8F88F4FF0000927E0009800F06C
:1010A000800028B1394640460A9AFFF778FF09E0E8
:1010B0000A9808B9012000E000200246394640465F
:1010C000FFF76DFF00984006000E0090781CC7B235
:1010D000A7EB0A00A04205D1574608F1010000F035
:1010E000FF0806E009F1010000F0FF09B9F1080F5F
:1010F000D4DB00BF681CC5B25D45AEDB00BFC8E7EE
:10110000F8B506460F4615461C4621E004EBD4719F
:101110004910C1F18001B14202DA00263819C7B284
:10112000C4F14000B84204DA002006460746FFF743
:101130008CFB012000902A78234639463046FFF781
:1011400060FF204604EBD07106EB6101CEB26D1C4E
:1011500028787E2802DC28782028D7DAF8BD70B5F8
:1011600000241BE004F1B0000021FFF7FAFA00218F
:101170000846FFF7F6FA00211020FFF7F2FA0025E3
:1011800008E03E4901EBC501085D0121FFF7E9FADE
:10119000681CC5B2802DF4DB601CC4B2082CE1DBF6
:1011A00070BD2DE9F04706460F4690469946DDF89A
:1011B00020A034460CE03D4606E052462946204633
:1011C000FFF77BFD681CC5B24D45F6DD601CC4B25F
:1011D0004445F0DDFFF73AFDBDE8F0872DE9F04129
:1011E00007460D469046002629463846FFF7FDFA89
:1011F000002403E0701CC6B2601CC4B2102CF9DBE2
:10120000681CC1B23846FFF7F0FA002403E0701CF6
:10121000C6B2601CC4B2102CF9DBBDE8F0812DE928
:10122000F05F81460F4614462046E21704EB5272E7
:10123000D2102146E31704EB5373DB10A4EBC30376
:101240000BB1012300E000231A44624302F0FF08BF
:1012500099F8006009F1010081460578812E05DBCF
:10126000402D03DBFF2D01D0FF2E1AD14FF0000AD5
:1012700013E000002C0100208805002088010020D8
:10128000987E00080C830008FC880008002007F8FE
:10129000010B0AF1010000F0FF0AC245F6DBBDE8D0
:1012A000F09F7F2D03DAA5F14000C5B202E0A5F161
:1012B0004100C5B2A6F18100C6B2BE2000FB0650B7
:1012C00000FB08FB0C2C04D0102C08D0182C0FD1DC
:1012D0000DE042465946384602F061F908E065489B
:1012E0000BEB00014246384602F059F900E000BF1E
:1012F00000BF00BFD3E72DE9F04F93B006460D467F
:1013000090461C46AA462046E21704EB5272D210C1
:101310002146E31704EB5373DB10A4EBC3030BB1BB
:10132000012300E000231A44624302F0FF0B0C2C5F
:1013300006D0102C04D0182C02D013B0BDE8F08FCA
:10134000224669464046FFF76AFF00272EE01DF857
:10135000070012904FF0000922E0129800F0800080
:1013600028B1E9B2F0B20122FFF7A7FC06E01C9811
:1013700020B9E9B2F0B20022FFF79FFC12984006B4
:10138000000E1290681C85B2A5EB0A00A04203D1A2
:101390005546701C86B206E009F1010000F0FF0915
:1013A000B9F1080FD9DB00BF781CC7B25F45CEDBAF
:1013B00000BFC2E72DE9FC5F07460D4691469A46FD
:1013C000DDE90C64B846AB46002001904BE0019883
:1013D00070BB3078802802DD0120019043E004EBEF
:1013E000D47108EB0902A2EB6101B94202DA2819B3
:1013F00085B247460BEB0A00001BA84200DA35E035
:1014000030780D2804D1281985B24746761C07E0AC
:10141000012000903278E9B2F8B22346FFF7F1FDDF
:10142000761C204604EBD07107EB61018FB21AE005
:101430000020019008EB0900001BB84202DA2819CD
:1014400085B247460BEB0A00001BA84200DA0DE00C
:10145000002023463246294600903846FFF74BFFCE
:10146000B61C381987B230780028B0D100BFBDE86B
:10147000FC9F000060C4080070B50346FA4C246865
:1014800034B1012C02D0022C06D103E0002205E089
:10149000082203E0182201E0102200BF00BF1A4416
:1014A000910200200CE0C0F10E050124AC400C407C
:1014B0002CB1C0F1040540F23754AC406140401CEF
:1014C0000528F0DB01EB822145F212446140002047
:1014D00009E0012484400C400CB1302500E02025B7
:1014E000E24C2554401C0528F3DD01F040040CB10A
:1014F000302500E02025DE4C84F8EF5101F0800417
:101500000CB1302500E02025D94C84F8F05101F4CD
:1015100080740CB1302500E02025D54C84F8B351FF
:10152000092010E0012484400C400CB1302400E07C
:101530002024C0F10E0505EB4506C6EB8515CC4E03
:1015400035442C72401C0E28ECDD002012E00124F2
:1015500084400C400CB1302500E02025C54C2468A7
:10156000641E241A04EB4406C6EB8414C04E3444B3
:101570002572401C0728EADD3026BE4C2468083C52
:10158000BA4D2E5508200DE0012484400C400CB1CA
:10159000302500E02025B74C24680F3C2618B34CBA
:1015A000A555401C0E28EFDD70BDF0B502460020A9
:1015B000C8E00021C0E001EB4103C3EB8113AC4C58
:1015C00023441B5C03F02003002B75D1072A78D23B
:1015D000DFE802F004101C2733465B00431803EBDE
:1015E000D3746410A3EB44040CB9012400E000247C
:1015F00025467FE0034600EBD3746410A0EB44045F
:101600000CB9012400E00024254673E0032391FB7C
:10161000F3F403FB14130BB9012300E000231D4670
:1016200068E04318032493FBF4F604FB16330BB96C
:10163000012300E000231D465CE0032691FBF6F643
:10164000044600EBD47706EB670303EBD376761002
:10165000A3EB46060EB9012600E00026354649E018
:1016600000FB01F4032694FBF6F706FB174600FB8C
:1016700001F303EBD3746410A3EB440434440CB9BA
:10168000012400E00024254634E000FB01F6032796
:1016900096FBF7FC07FB1C6700FB01F404EBD47618
:1016A0007610A4EB4606BB1903EBD3767610A3EBBA
:1016B00046061EB9012602E03DE002E0002635465E
:1016C00018E000FB01F6032796FBF7FC07FB1C66FE
:1016D000441804EBD4777F10A4EB4707F31903EB0E
:1016E000D3767610A3EB46060EB9012600E000265D
:1016F000354600BF00BF01EB4103C3EB81135C4CD7
:1017000023441B5C03F0FE0401EB4103C3EB811394
:10171000574E33441B5C03F00203012B01DD012310
:1017200000E000236B40234301EB4104C4EB811430
:101730004F4E34442354491C4E4B1B689942FFF6CC
:101740003AAF401C4B4B1B689842FFF632AFF0BDDE
:101750002DE9F0410020002400223CE0002134E08B
:1017600001264B1C26E002EB4207C7EB8217DFF88D
:1017700000C167447F5C07F011070FB9012700E043
:10178000002702EB420CCCEB821CDFF8E480C4445F
:101790001CF803C00CF0110CBCF1000F02D14FF08B
:1017A000010C01E04FF0000C674501D1761C00E010
:1017B00004E05B1C2F4F3F68BB42D4DB00BF052E0B
:1017C00001DBB71E3844591E491C2A4E3668361FA5
:1017D0008E42C5DC521C274E3668B242BEDB002268
:1017E0003CE0002134E001264B1C26E001EB4107E0
:1017F000C7EB8117DFF878C06744BF5C07F01107BB
:101800000FB9012700E0002703EB430CCCEB831C4E
:10181000DFF85C80C4441CF802C00CF0110CBCF171
:10182000000F02D14FF0010C01E04FF0000C6745B2
:1018300001D1761C00E004E05B1C0E4F3F68BB4208
:10184000D4DB00BF052E01DBB71E3844591E491CEE
:10185000084E3668361F8E42C5DC521C054E36686F
:10186000B242BEDB00226EE03C0100207007002087
:10187000880500202C01002000215EE002EB4206DA
:10188000C6EB8216FE4F3E44765C06F011060EB99A
:10189000012700E00027561C06EB460CCCEB861611
:1018A000DFF8DCC36644765C06F011060EB901264B
:1018B00000E00026B7423FD102EB4206C6EB82169B
:1018C000EF4F3E44765C06F011060EB9012700E0AA
:1018D000002702EB4206C6EB8216DFF8A4C3B4442D
:1018E0004E1C1CF8066006F011060EB9012600E039
:1018F0000026B74220D102EB4206C6EB8216E04F2B
:101900003E44765C06F011060EB9012700E0002780
:10191000561C06EB460CCCEB8616DFF864C3B444C9
:101920004E1C1CF8066006F011060EB9012600E0F8
:101930000026B74200D1C01C491CD24E3668761E24
:101940008E429BDC521CCF4E3668761E964293DC4C
:101950000022D2E00021C9E059B102EB4206C6EBF9
:101960008216C74F37444E1EBE5D06F01106002E8C
:1019700076D102EB4206C6EB8216C14F3E44765C3E
:1019800006F01106002E6BD002EB4206C6EB821663
:1019900037444E1CBE5D06F01106002E60D102EBEE
:1019A0004206C6EB8216B64F37448E1CBE5D06F06B
:1019B0001106002E54D002EB4206C6EB8216B04F41
:1019C0003744CE1CBE5D06F01106002E48D002EB57
:1019D0004206C6EB8216AA4F37440E1DBE5D06F0C6
:1019E0001106EEB302EB4206C6EB8216A44F374453
:1019F0004E1DBE5D06F0110696BB02EB4206C6EB1D
:101A000082169F4F37448E1DBE5D06F011063EB311
:101A10009C4E3668F61F8E420AD002EB4206C6EB99
:101A20008216974F3744CE1DBE5D06F01106BEB933
:101A300002290ADB02EB4206C6EB8216904F3744BE
:101A40008E1EBE5D06F01106DEB903290CDB02EB2B
:101A50004206C6EB82168A4F3744CE1EBE5D00E0BA
:101A600043E006F0110666B904293DDB02EB4206AD
:101A7000C6EB8216824F37440E1FBE5D06F011067C
:101A800096B3804E3668083E8E420BDD02EB42066E
:101A9000C6EB82167A4F374401F10806BE5D06F0A8
:101AA000110616BB774E3668093E8E420BDD02EBFF
:101AB0004206C6EB8216724F374401F10906BE5D3D
:101AC00006F011068EB96F4E36680A3E8E420BDD67
:101AD00002EB4206C6EB8216694F374401F10A0653
:101AE000BE5D06F0110606B92830491C654E366801
:101AF000B61F8E423FF730AF521C624E3668B2427C
:101B0000FFF628AF0022D7E00021CEE059B14E1EEB
:101B100006EB4607C7EB8616594F3E44B65C06F007
:101B20001106002E60D101EB4106C6EB8116544F21
:101B30003E44B65C06F01106002E55D04E1C06EB56
:101B40004607C7EB86164E4F3E44B65C06F01106BC
:101B5000002E49D18E1C06EB4607C7EB8616484F70
:101B60003E44B65C06F01106F6B3CE1C06EB460703
:101B7000C7EB8616424F3E44B65C06F011069EB394
:101B80000E1D06EB4607C7EB86163D4F3E44B65C7E
:101B900006F0110646B34E1D06EB4607C7EB861648
:101BA000374F3E44B65C06F01106EEB98E1D06EBCB
:101BB0004607C7EB8616324F3E44B65C06F0110668
:101BC00096B1304E3668F61F8E420AD0CE1D06EB17
:101BD0004607C7EB86162A4F3E44B65C06F0110650
:101BE00016B902290CDB00E05EE08E1E06EB46070C
:101BF000C7EB8616224F3E44B65C06F01106CEB9FE
:101C000003290ADBCE1E06EB4607C7EB86161C4FE0
:101C10003E44B65C06F0110666B9042943DB0E1F8C
:101C200006EB4607C7EB8616154F3E44B65C06F03A
:101C300011064EB3134E3668083E8E420BDD01F19D
:101C4000080606EB4607C7EB86160D4F3E44B65C0A
:101C500006F0110646BB0B4E3668093E8E420BDD80
:101C600001F1090606EB4607C7EB8616044F3E4412
:101C7000B65C06F01106BEB9024E36680A3E04E0B4
:101C8000880500202C0100200DE08E420BDD01F1C3
:101C90000A0606EB4607C7EB8616FE4F3E44B65CC7
:101CA00006F0110606B92830491CFB4E3668B61FEF
:101CB0008E423FF72BAF521CF74E3668B242FFF60A
:101CC00023AF002212E000210BE002EB4206C6EB3C
:101CD0008216F04F3E44765C06F0110606B9641C8D
:101CE000491CED4E3668B142EFDB521CEA4E3668B5
:101CF000B242E8DB64266643E74F3F687F4396FBCA
:101D0000F7F6C6F13206002E09DD64266643E24F7F
:101D10003F687F4396FBF7F6C6F1320509E064267B
:101D20006643DD4F3F687F4396FBF7F6C6F1320608
:101D30007542052695FBF6F606EB860600EB460097
:101D4000BDE8F081F0B5D44E30683668711E0122CE
:101D5000012500233DE0002438E000BF104452423A
:101D6000002A13DA2944002903DBCB4E3668B1423E
:101D70000CD1002901DA002602E0C74E3668761E33
:101D800031466D42801E062800D1401E00EB400601
:101D9000C6EB8016BF4F3E44765C06F02006002E50
:101DA000DCD1BE4EF65CC4F1070C012707FA0CF734
:101DB0003E400EB1022600E0002600EB4007C7EBD4
:101DC0008017DFF8D0C267447E54641C082CC4DB43
:101DD0005B1CB34E3668B342BDDBF0BD70B5024646
:101DE00002EB4204C4EB8214AA4D2C44645C04F060
:101DF000200404B170BD921E891E002019E000234A
:101E000014E0A84C245CC3F104060125B5402C4025
:101E10000CB1302400E02024D51805EB4506C6EBB4
:101E200085159C4E35440E18AC555B1C052BE8DB24
:101E3000401C0528E3DB00BFDCE730B59A4B1B688C
:101E4000062B00DC30BD984B1B681A0300200CE009
:101E5000C0F111040123A34013402BB1C0F10504CC
:101E600041F62573A3405A40401C0628F0DB8E4BF8
:101E70001B6802EB0332002025E0002120E000EB8C
:101E800040035C180123A34013400BB1302400E051
:101E9000202400EB4003C3EB80137E4D1D447E4B9A
:101EA0001B680B3B0B44EC547B4B1B680B3B0B44FC
:101EB00003EB4305C5EB8313764D2B441C54491C9F
:101EC0000329DCDB401C0628D7DB00BFBAE770B56E
:101ED00002460B46002019E0002114E0734C245CFC
:101EE000C1F106060125B5402C400CB1302400E0BC
:101EF0002024551805EB4506C6EB8515654E35447F
:101F00001E18AC55491C0729E8DB401C0728E3DBF9
:101F100070BD30B500210846FFF7D9FF5E4909685A
:101F2000C81F0021FFF7D3FF5B480068C11F0020D6
:101F3000FFF7CDFF00242FE020215D48015504EB81
:101F40004400C0EB8410534A1044C17152480068E9
:101F50000838204400EB4002C2EB80104D4A104488
:101F6000C1714D480068083800EB4002C2EB801098
:101F7000484A1044015548480068083802194C483E
:101F8000815404EB4400C0EB8410424A02444248AE
:101F9000006808381154641C082CCDDB00240BE0C9
:101FA000202143483D30015504EB4400C0EB841030
:101FB000384A10440172641C092CF1DB002413E040
:101FC0002021354800680838021939483D308154CD
:101FD000314800680838204400EB4002C2EB801012
:101FE0002C4A10440172641C082CE9DBFFF725FF22
:101FF000002447E02C49096801EB810202EB411102
:102000002C4A02EB41010E3131F814000621FFF792
:10201000E5FE2548006800EB800202EB4010254AEF
:1020200002EB40000E3030F814100620FFF7D6FE09
:1020300000251AE01C4A126802EB820303EB4212ED
:102040001C4B03EB42020E3232F81510164A12688E
:1020500002EB820303EB4212164B03EB42020E32F9
:1020600032F81400FFF7BAFE6D1C0F48006800EB51
:10207000800101EB40100F4901EB40008089A8422C
:10208000D8DC641C0848006800EB800101EB4010BC
:10209000084911E0880500202C010020C11800200B
:1020A0003801002053010020400100204C01002095
:1020B000330700205896000801EB40008089A042B9
:1020C00098DC08241DE0204604EBD0714910A4EBF5
:1020D000410109B9302100E0202104EB4402C2EBA8
:1020E0008412FE4B1A449171204604EBD0714910C2
:1020F000A4EB410109B9302200E02022F8490A5539
:10210000641CF84800680938A042DCDA30BD2DE9CB
:10211000F04140F68961F14803F099FEFFF7F9FEBE
:10212000FFF710FEF0480068401C00BB0020EE499D
:10213000086008460068FFF738FAEB480068FFF7C8
:102140009BF9FFF705FB074601240EE02046FFF749
:102150002CFA2046FFF790F9FFF7FAFA0646BE423E
:1021600002DA3746E0480460641C072CEEDDDE48E6
:102170000068FFF71AFADC480068FFF77DF90024D1
:102180001BE0002514E004EB4400C0EB8410D349AD
:102190000844405D00F0110008B1012000E000207B
:1021A00004EB4401C1EB8411CC4A114448556D1C29
:1021B000CC4800688542E6DB641CCA48006884425B
:1021C000DFDBBDE8F0812DE9F0410346002434E077
:1021D0001D783DB31E78C54FBD5D002015E0C44F8E
:1021E00057F822703F5C2F444FF0FF0C97FBFCF830
:1021F0000CFB1877FEB2471CDF5DDFF8F8C21CF855
:1022000006C087EA0C071F54401C9042E7DB1046CB
:1022100003E0461C9E5D1E54401C8E18761E8642AE
:10222000F7DC09E0002003E0451C5D5D1D54401C07
:102230008D186D1E8542F7DC641C8C42C8DBBDE83E
:10224000F081F0B503460D46581C18B19818B0F54A
:10225000486F02DD4FF0FF30F0BD002124E0501A3E
:10226000401E012404FA00F02840E0B15818C617B7
:1022700000EB5676F610A04FBE5D5C18E71704EB36
:102280005777FF10A4EBC707C7F1070C012707FA20
:102290000CF73E435818C71700EB5777FF10DFF8CD
:1022A00058C20CF80760491C9142D8DB9818D3E754
:1022B000014648F24010814208DB49F6FC70814239
:1022C00004DCA1F50140403881B202E001F57B5009
:1022D00081B2C8B20A1202EB420200EB821080B255
:1022E00070470146302905DB392903DCA1F13000B4
:1022F000C0B27047412905DB5A2903DCA1F1370040
:10230000C0B2F6E7202901D12420F2E7242901D127
:102310002520EEE7252901D12620EAE72A2901D147
:102320002720E6E72B2901D12820E2E72D2901D13A
:102330002920DEE72E2901D12A20DAE72F2901D131
:102340002B20D6E72C20D4E7F0B50446002324B197
:10235000012C1CD0022C37D12FE0032091FBF0F58B
:102360006648805C001D0A2606FB0503032091FBDE
:10237000F0F500FB1510012802D0022804D101E07D
:102380001B1D02E0DB1D00E000BF00BF23E008468C
:1023900001EBD07677105A4EB65C361D4FF00B0C21
:1023A0000CFB07660D4601EBD5777F10A1EB4707C5
:1023B0004FF0060C0CFB07630DE05248805C001DDB
:1023C000082505FB010306E04F48805C001D0D2534
:1023D00005FB010300BF00BF1846F0BD01463029D0
:1023E00003DB392901DC01207047412903DB5A292D
:1023F00001DC0120F8E720290FD024290DD0252960
:102400000BD02A2909D02B2907D02D2905D02E2918
:1024100003D02F2901D03A2901D10120E4E700207F
:10242000E2E70146302903DB392901DC012070474E
:102430000020FCE70246812A01DB9F2A03DDE02A17
:102440000FDBEB2A0DDC40290BDB9F2A01D1FC2995
:1024500003DCEB2A03D1BF2901DD002070470120F6
:10246000FCE70020FAE72DE9F74F86B007469246D1
:102470000024A0464FF4C871244803F0E8FC002073
:102480000546234908605DE00798401EA84207DD25
:102490006A1CB95C785DFFF7CDFF08B103230CE03F
:1024A000785DFFF7BEFF08B1002306E0785DFFF717
:1024B00095FF08B1012300E002230DB91548037010
:1024C000144813490968405C984206D010480068D7
:1024D000401C0F4908600F490B541DE0880500207F
:1024E000F60600202C0100204801002032A300083D
:1024F0001800002032A2000811140020DEA80008F5
:10250000E1A80008E4A80008E7A8000831170020A7
:1025100034010020A1150020FD48FE490968405CF7
:10252000401CC1B2FA48FB4A12688154032B08D1FF
:10253000F8490968405C401CF549F64A126888541D
:102540006D1C6D1C079885429EDBF2480068401C9C
:10255000F049086060E100200190EF48005D20B97B
:10256000ED49601C085C012808D0EB48005D01289B
:102570007ED1E949601C085C0028F9D1E44A115D6C
:10258000E54A105D5246FFF7DFFE8346E04B621CD2
:10259000995CE14B985C5246FFF7D6FE0BEB0001CD
:1025A0000591DB48025D0346601C185C1118524619
:1025B0000120FFF7C9FE81460599494558DD012CE8
:1025C00027DB601ED449085C022822D1601ED04A55
:1025D000105C125D811852460220FFF7B5FE83465B
:1025E000CB4B621C995CCC4B985C5246FFF7ACFE1F
:1025F00058440390601EC64A115C52460220FFF701
:10260000A3FE00EB09010398814204DA0020039045
:1026100001E000200390BF480068801EA0422ADD30
:10262000BD49A01C085C022825D1B94A115DBA4AEF
:10263000105D5246FFF788FE8346B54A601C125C67
:10264000B34BA01C185C111852460220FFF77CFE09
:1026500058440290AE4AA01C115C52460220FFF77B
:1026600073FE00EB09010298814206DA002000E0C7
:10267000D0E0029001E000200290039858B1029847
:1026800048B1DDE90210884202DA4FF0FF3000E085
:10269000012001900AE0039810B14FF0FF3004E0F0
:1026A000029808B1012000E0002001900198E8B3F1
:1026B0000198401CD0B9601E9549085C095D08442A
:1026C000C1B2601E924A1154254609E09249681C25
:1026D000095C914841558E49681C085C48556D1C41
:1026E0008C480068401EA842F0DC1CE002218A4AA7
:1026F000601C11548649095C854AA01C105C084482
:10270000C1B2601C1154A51C08E08349681C085C18
:1027100048557F49681C085C48556D1C7D48006819
:10272000401EA842F1DC7B48006800E003E0401E48
:10273000784908606DE077480068801EA04223DD7C
:102740007549A01C085C01281ED17149601C095CF8
:102750006F4AA01C105C0844C1B2601C1154A51C37
:1027600008E06D49681C085C48556949681C085CAC
:1027700048556D1C67480068401EA842F1DC65485A
:102780000068401E634908600121634801556048A4
:10279000015D0246601C105C084411460855651C2A
:1027A00008E05D49681C085C48555949681C085C8C
:1027B00048556D1C57480068401EA842F1DC55483A
:1027C0000068401E53490860012C22DB601E5249FC
:1027D000085C01281DD1601E4D49085C095D084454
:1027E000C1B2601E4A4A1154254608E04A49681C95
:1027F000085C48554649681C085C48556D1C4548AE
:102800000068401EA842F1DC42480068401E414971
:10281000086001E0641C00BF3E480068401EA04202
:102820003FF799AE0024BBE0394A115D3A4A105D8A
:102830005246FFF789FD8346354B621C995C364B47
:10284000985C5246FFF780FD584405903048025D81
:102850000346601C185C111852460220FFF774FDF5
:102860008146012C0ADB601E2B49085C022805D139
:102870002A4810F80A00001DA9EB00092548006845
:10288000801EA0420ADD2449A01C085C022805D154
:10289000224810F80A00001DA9EB000905984845D8
:1028A0007CDD012C23DB601E1B49085C02281ED145
:1028B000601E1749085C095D0844C1B2601E144AD5
:1028C0001154254608E01449681C085C4855104915
:1028D000681C085C48556D1C0E480068401EA842E4
:1028E000F1DC0C480068401E0A490860641E094873
:1028F0000068801EA0422CDD0749A01C085C02284D
:1029000027D10349601C095C014AA01C105C07E048
:102910003117002034010020A1150020E4A8000890
:102920000844C1B2601C1154A51C08E0FD49681C94
:10293000085C4855FC49681C085C48556D1CFB4800
:102940000068401EA842F1DCF8480068401EF749C4
:1029500008600220F3490855F348015D0246601CF7
:10296000105C084411460855651C08E0ED49681CD8
:10297000085C4855EC49681C085C48556D1CEB48E0
:102980000068401EA842F1DCE8480068401EE749A4
:102990000860012C00DB641E02E0FFE7641C00BF3E
:1029A000E2480068401EA0423FF73EAF0020E049E9
:1029B00008604FF4C871DF4803F049FA00252BE1A5
:1029C000D848405DC8BB04220121D9480068FFF700
:1029D00038FCD7490860D84810F80A20D248415D31
:1029E000D3480068FFF72DFCD1490860002656E067
:1029F000CD48405D801EB04220DD08EB0600385C0B
:102A000030386421484308EB0601491C795C3039B1
:102A100001EB810100EB410108EB0600801C385CF2
:102A20003038084480B204900A22C14804990068F2
:102A3000FFF707FCBE49086030E038E0BA48405D67
:102A4000801EB04217D108EB0600401C385C3038BD
:102A500008EB0601795C303901EB810100EB4100A4
:102A600080B204900722B24804990068FFF7E9FB9E
:102A7000AF49086012E0AC48405D401EB0420DD145
:102A800008EB0600385C303880B204900422A84875
:102A900004990068FFF7D5FBA5490860F61CA24819
:102AA000405DB042A4DCA048405D8044B3E09D4856
:102AB000405D01284AD1042202219D480068FFF7A9
:102AC000C0FB9B4908609D4810F80A209648415D6C
:102AD00097480068FFF7B5FB9549086000262DE090
:102AE0009148405D401EB04219DD08EB0601785C5C
:102AF000FFF7F7FBC0EB001000EB400208EB06010C
:102B0000491C785CFFF7EDFB104404900B228848C9
:102B100004990068FFF795FB854908600DE008EB14
:102B20000601785CFFF7DDFB0490062280480499DB
:102B30000068FFF786FB7E490860B61C7A48405D56
:102B4000B042CDDC7848405D804464E07548405D2B
:102B5000022827D10422114675480068FFF771FB4F
:102B600073490860764810F80A206F48415D704844
:102B70000068FFF766FB6E49086000260AE008EB74
:102B80000600395C08226A480068FFF75AFB68496A
:102B90000860761C6448405DB042F0DC6248405DED
:102BA000804438E00422082161480068FFF749FBAF
:102BB0005F4908605C4810F805B00BEBDB70411012
:102BC000604810F80A205A480068FFF73AFB584955
:102BD0000860002615E008EB4601491C795C08EB0B
:102BE0004602BA5C01EB022188B2FFF761FB834623
:102BF0000D2259464E480068FFF723FB4C490860F8
:102C0000761C4949485D00EBD071B6EB610FE2DB01
:102C10004548405D80446D1C44480068854205DAA3
:102C200043480068401C00287FF4CAAE4048006852
:102C3000401C18B1012009B0BDE8F08F0020FAE770
:102C40002DE9F04706460F4690461B2E01DB022079
:102C500004E00A2E01DB012000E0002081464D4601
:102C60007AE02A4641463846FFF7FDFB002872D03D
:102C7000EDB9012418E02E490968C81D04EB840150
:102C800001EB4411304A02EB4101091D2F4A126841
:102C900031F81210C21700EB5272B1EBE20F02DBF7
:102CA0002046BDE8F087641C092CE4DD53E0012DCB
:102CB0001CD10A2417E01E490968C81D04EB8401D1
:102CC00001EB4411204A02EB4101091D1F4A126821
:102CD00031F81210C21700EB5272B1EBE20F01DBB8
:102CE0002046DEE7641C1A2CE5DD34E0022D32D1EB
:102CF0001B242EE00E490968C81D04EB840101EB7A
:102D00004411114A02EB4101091D104A126831F8C1
:102D10001210C21700EB5272B1EBE20F18DB204623
:102D2000BFE70000A115002031170020340100206A
:102D30003001002011140020DEA80008E1A80008DE
:102D4000E4A80008E7A80008589600083C01002005
:102D5000641C282CCEDD6D1C022D82DD0020A0E736
:102D60002DE9F14F8CB001200B900A90EC200690D9
:102D70004FF00008002600200990F9490860F94941
:102D800008600998002801DD099802E00C9802F01B
:102D9000FDFF0890089818B900200DB0BDE8F08F2D
:102DA000089ADDE90B01FFF74BFF8246BAF1000FED
:102DB00001D10020F1E70B9818B9EB48C0F800A04A
:102DC0000EE00B98824503DCE7490B98086007E0AA
:102DD0000A9818B1E448C0F800A001E00020DCE740
:102DE000E148006800EB800101EB4010DF4901EB96
:102DF0004000001DDA49096830F81170DC480068AD
:102E0000C0EBC700042801DD042003E0D8480068B7
:102E1000C0EBC70007900798002807DD0021D448C1
:102E2000079A0068FFF70DFAD1490860D049096890
:102E3000C81DC11700EB5171CC100AE0CD490698AE
:102E400008550698EC2801D1112000E0EC200690EE
:102E5000641CBC42F2DBC448006800EB800101EB5B
:102E60004010C24901EB40004088C3490860084651
:102E70000168C24802F0EBFFBB48006800EB80012C
:102E800001EB4010B94901EB40001A30B449096820
:102E900001EB410130F811000590B348006800EBE8
:102EA000800101EB4010B14901EB40003230AC49E8
:102EB000096801EB410130F811100491DDE90410BB
:102EC00000EB010BA848006800EB800101EB40100B
:102ED000A64901EB40001A30A149096801EB410104
:102EE00000EB4100B0F804909F48006800EB8001BF
:102EF00001EB40109D4901EB4000323098490968D0
:102F000001EB410100EB41008088039000240FE0B9
:102F1000002509E0404608F101089649085C0BFBD2
:102F20000561964A50546D1C4D45F3DB761C641CBC
:102F300005988442ECDB00241CE0002515E04D459B
:102F400009DA404608F101088A49085C0BFB056173
:102F50008A4A505408E0404608F101088549085C57
:102F60000BFB0941854A50546D1C03988542E6DBF2
:102F7000761C641C04988442DFDB7B48006800EB0D
:102F8000800101EB4010794901EB40001A3074498F
:102F9000096801EB410100EB41004088A0EB09000A
:102FA00002907148006800EB800101EB40106F490E
:102FB00001EB400032306A49096801EB410100EB46
:102FC000410041880398081A01904FF0000800263C
:102FD00000241FE099216A4802F039FF654800EBA0
:102FE00008014A46664802F0F0FE49466448029AE3
:102FF000FFF7E9F8002507E06148405D0BFB05712C
:1030000031445E4A50546D1C02988542F4DBC8443A
:10301000761C641C05988442DCDB002420E09921A6
:10302000574802F014FF534800EB08015448039A34
:1030300002F0CBFE5248019A0399FFF7C4F800252D
:1030400007E04F48405D0BFB057131444B4A50543B
:103050006D1C01988542F4DB03988044761C641C47
:1030600004988442DBDB40480068112101EB8000BA
:1030700044490860FFF74BF801208EE60246A12A7A
:1030800001DBAA2A03DBB02A07DBFA2A05DCA12927
:1030900003DBFE2901DC012070470020FCE701462C
:1030A0004AF2A11081420EDB4AF6FE1081420ADC90
:1030B000C8B2A138A122C2EB212202EB420200EBEE
:1030C000421080B270474BF2A10081420EDB4FF6F6
:1030D000FE1081420ADCC8B2A138A622C2EB21222E
:1030E00002EB420200EB421080B2EBE7C8B2A1381B
:1030F000A622C2EB212202EB420200EB421080B278
:10310000E0E72DE9F04FC0B04FF0040C0226DFF8E5
:1031100074A0DAF800A09AFBF6F8DFF868A0DAF8F5
:1031200000A09AFBF6FB06FB1BA9DFF858A09AF853
:1031300000A00CFB0AFA0AF0FF070023A3E04FF0FF
:103140001B0A8DF800A04FF02A0A8DF801A08DF817
:1031500002704FF0000A8DF803A00420002184E0E3
:103160003C01002048010020400100205896000842
:10317000300100201114002038010020C118002067
:10318000511A00202C01002003FB06F201EB410A3A
:10319000CAEB811ADFF88CB1DA441AF802A0BAF14E
:1031A000010F11D101EB410ACAEB811AD34402F19C
:1031B000010A1BF80AA0BAF1010F05D14FF0FF0A6E
:1031C0000DF800A0401C40E001EB410ACAEB811A57
:1031D000DFF850B1DA441AF802A0BAF1010F11D1A8
:1031E00001EB410ACAEB811AD34402F1010A1BF830
:1031F0000AA0BAF1000F05D14FF0F00A0DF800A0B7
:10320000401C22E001EB410ACAEB811ADFF814B13D
:10321000DA441AF802A0BAF1000F11D101EB410A09
:10322000CAEB811AD34402F1010A1BF80AA0BAF1D1
:10323000010F05D14FF00F0A0DF800A0401C04E06B
:103240004FF0000A0DF800A0401C921C002407E07B
:10325000A0F1010A1DF80AA00DF800A0401C641C92
:10326000ACF1010AA245F3DC491CDFF8BCA0DAF896
:1032700000A0514588DB002500E06D1C07F1040A21
:103280005545FADB5B1C4345FFF659AFB9F1000F1A
:1032900045D04FF01B0A8DF800A04FF02A0A8DF898
:1032A00001A08DF802704FF0000A8DF803A00420F1
:1032B000002127E008FB06F301EB410ACAEB811A63
:1032C000DFF860B0DA441AF803A0BAF1010F05D1B3
:1032D0004FF0F00A0DF800A0401C04E04FF0000A87
:1032E0000DF800A0401C002407E0A0F1010A1DF821
:1032F0000AA00DF800A0401C641CACF1010AA24514
:10330000F3DC491CDFF820A0DAF800A05145D1DB3E
:10331000002500E06D1C07F1040A5545FADB40B0BA
:10332000BDE8F08F880500202C01002008B50121A0
:103330001C2001F0C7F84FF4A040ADF800001020A9
:103340008DF8030003208DF8020069460F4800F055
:10335000FDFD0220ADF8000010208DF803000320D1
:103360008DF8020069460A4800F0F0FD4FF4005065
:10337000ADF8000010208DF8030003208DF8020046
:103380006946044800F0E2FD08BD0000000C014061
:10339000000801400010014070B50546002405E01A
:1033A000601CC4B2C82C01DD002070BD02213A4867
:1033B00001F03BFA0028F3D02946374801F0E2F942
:1033C000002405E0601CC4B2C82C01DD0020ECE73D
:1033D0000121314801F029FA0028F3D02E4801F0EC
:1033E000D3F9C0B2E1E700B587B00121082001F0B0
:1033F00069F80121880301F072F84FF46040ADF8DC
:10340000180018208DF81B0003208DF81A0006A95B
:10341000224800F09BFD4FF46041204800F043FE3D
:103420000020ADF804004FF48270ADF806000020D3
:10343000ADF808000220ADF80A000120ADF80C003C
:103440004002ADF80E003820ADF810000020ADF8B5
:1034500012000720ADF8140001A90F4801F0BCF8D4
:1034600001210D4801F05DF9FF20FFF795FF07B03E
:1034700000BD10B50446084800884FF6C7710840E3
:103480000549088008460088204308800121024839
:1034900001F047F910BD000000380040000C014069
:1034A00010B500240020D14908609020FFF774FF78
:1034B0000020FFF771FF0020FFF76EFF0020FFF7ED
:1034C0006BFFFF20FFF768FF44EA0024FF20FFF7AF
:1034D00063FF04430120C649C1F8B001204610BD76
:1034E00008B50121082000F0EDFF4FF48050ADF841
:1034F000000010208DF8030003208DF802006946BB
:10350000BC4800F023FD4FF48051BA4800F0CBFDD9
:103510000120B6490860FFF766FF0020FFF7A9FF0A
:10352000FFF7BEFFB449088008BD10B50024002095
:10353000AE4908600520FFF72FFFFF20FFF72CFFA3
:1035400004460120AA49C1F8B001204610BD10B5BB
:1035500004460020A54908600120FFF71DFF204612
:10356000FFF71AFF0120A249C1F8B00110BD10B544
:1035700000209E4908600620FFF70EFF01209C49AD
:10358000C1F8B00110BD10B50020984908600420B2
:10359000FFF702FF01209649C1F8B00110BD2DE9E7
:1035A000F04106460C46174600209049086003206B
:1035B000FFF7F2FEC4F30740FFF7EEFEC4F3072067
:1035C000FFF7EAFEE0B2FFF7E7FE002505E0FF2087
:1035D000FFF7E2FE7055681C85B2BD42F7DB0120A3
:1035E00082490860BDE8F08110B500BFFFF79DFF7C
:1035F00000F001000028F9D110BD2DE9F041064688
:103600000C461746FFF7B3FF0020784908600220F8
:10361000FFF7C2FEC4F30740FFF7BEFEC4F3072066
:10362000FFF7BAFEE0B2FFF7B7FE002504E0705DD9
:10363000FFF7B2FE681C85B2BD42F8DB01206B4982
:103640000860FFF7D1FFBDE8F0812DE9F0410746A2
:103650000E461446F0B2C0F58075AC4200DC25463B
:1036600012E02A4631463846FFF7C7FFAC4200D188
:103670000BE02F442E44601B84B2B4F5807F02DD42
:103680004FF4807500E02546EBE700BFBDE8F08110
:1036900010B50446214659A002F022FA2403FFF790
:1036A00066FFFFF7A1FF0020504908602020FFF7C8
:1036B00073FEC4F30740FFF76FFEC4F30720FFF764
:1036C0006BFEE0B2FFF768FE01204949C1F8B00186
:1036D000FFF78AFF10BD2DE9F05F81460F461646C1
:1036E000DFF820B14FEA1738C7F30B0ACAF5805448
:1036F000A64200DC344644E04FEA08314FF48052E1
:103700005846FFF74CFF002508E00AEB05001BF8C0
:103710000000FF2800D003E0681C85B2A542F4DB5E
:1037200000BFA54216DA4046FFF7B2FF002507E0CA
:1037300019F8050005EB0A010BF80100681C85B2B9
:10374000A542F5DB4FEA08314FF480525846FFF7A7
:103750007CFF04E0224639464846FFF776FFA64242
:1037600000D10FE008F101084FF0000AA1442744FE
:10377000301B86B2B6F5805F02DD4FF4805400E066
:103780003446B9E700BFBDE8F09F10B5FFF7EFFE84
:10379000FFF72AFF002015490860C720FFF7FCFD4E
:1037A00001201349C1F8B001FFF71EFF10BD10B58D
:1037B00000200E490860B920FFF7EEFD01200C49FA
:1037C000C1F8B001032000F038F810BD10B500209A
:1037D00006490860AB20FFF7DFFD01200449C1F86E
:1037E000B001032000F029F810BD0000B081214293
:1037F00000802142000C01405801002066653A25F6
:10380000780D0A00EA1A002010B56FF0040000F0ED
:103810001EFB2E4800682E49B0FBF1F02D490870C0
:103820000846007800EB4001C1EBC0104FF6FF7175
:1038300001EAC0002849088010BD0146254A1278D7
:103840004A434FF0E0235A6100229A611A461269F6
:1038500042F001021A6100BF4FF0E022106900F04F
:1038600001021AB100F48032002AF5D04FF0E022B4
:10387000126922F001024FF0E0231A6100229A61DE
:1038800070470146144A12884A434FF0E0235A61B8
:1038900000229A611A46126942F001021A6100BFC1
:1038A0004FF0E022106900F001021AB100F48032FA
:1038B000002AF5D04FF0E022126922F001024FF009
:1038C000E0231A6100229A61704700000400002082
:1038D00000127A005A0100205C010020014600BF5E
:1038E000704700BFFA4A128802F04002002AF9D05D
:1038F000C2B2F74B1B1D1A80704710B586B0044644
:10390000012144F2040000F0DDFD4FF40070ADF839
:10391000140003208DF8160018208DF8170005A953
:10392000EC4800F013FB4FF48060ADF81400042065
:103930008DF8170005A9E74800F008FB25208DF851
:10394000000003208DF801008DF8020001208DF8A1
:103950000300684600F031FA01940020ADF8080039
:10396000ADF80A00ADF80C00ADF810000C20ADF871
:103970000E0001A9D64800F0D2FF012240F22441F6
:10398000D34801F064F8012240F22551D04801F0FB
:103990005EF80121CE4801F04EF806B010BD10B51A
:1039A00086B004460121880400F099FD0121082019
:1039B00000F088FD27208DF8040000208DF8050018
:1039C0008DF8060001208DF8070001A800F0F5F938
:1039D0004FF48060ADF8000003208DF8020018203D
:1039E0008DF803006946BC4800F0B0FA4FF400605F
:1039F000ADF8000004208DF803006946B64800F0D9
:103A0000A5FA02940020ADF80C00ADF80E00ADF858
:103A10001000ADF814000C20ADF8120002A9AF4858
:103A200000F07DFF012240F22441AC4801F00FF884
:103A3000012240F22551A94801F009F80121A748C7
:103A400000F0F9FF06B010BD10B586B004460121A4
:103A5000480400F044FD0121042000F033FD04205F
:103A6000ADF8140003208DF8160018208DF817000B
:103A700005A9984800F06AFA0820ADF8140004205F
:103A80008DF8170005A9934800F060FA0194002012
:103A9000ADF80800ADF80A00ADF80C00ADF8100064
:103AA0000C20ADF80E0001A98D4800F038FF26204B
:103AB0008DF8000002208DF8010000208DF8020032
:103AC00001208DF80300684600F077F9012240F2EA
:103AD0002551834800F0BBFF012240F22441804879
:103AE00000F0B5FF01217E4800F0A5FF06B010BD33
:103AF00000BF7B49098801F040010029F9D07849CD
:103B0000091D0880704770B504460D4600217548B0
:103B100001F0F6FC04E014F8010BFFF7E9FF6D1E5D
:103B2000002DF8DC01216F4801F0EAFC70BD00BFF8
:103B30006A49098801F040010029F9D06749091D47
:103B40000880704770B504460D460021654801F0B5
:103B5000D7FC04E014F8010BFFF7E9FF6D1E002D00
:103B6000F8DC01215F4801F0CBFC70BD00BF584973
:103B7000098801F040010029F9D05549091D088044
:103B8000704770B504460D460021564801F0B8FC58
:103B900004E014F8010BFFF7E9FF6D1E002DF8DCBF
:103BA0000121504801F0ACFC70BD70B5002440F21A
:103BB00025514B4801F030F8A0B1494800F0ACFF66
:103BC000C4B249480068632804D248484649096895
:103BD000445402E000204449086043480068401C07
:103BE0004149086040F224413D4801F015F868B1B0
:103BF0003B480088C5B23A48001D0088C5B2002085
:103C0000394908606421394802F021F970BD2DE975
:103C1000F04781460F46154698460024002629465F
:103C2000484602F0A1F80446284602F0AFF82044C6
:103C300000F1010A4146504602F096F8064614B1DA
:103C40000EB1B44202D90020BDE8F087284602F048
:103C50009DF80444321B2146384602F01AF901202F
:103C6000F2E770B5002440F225511C4800F0D4FF63
:103C7000B8B11A4800F050FFC4B21D480068772858
:103C800004D21C481A490968445402E0002018492B
:103C9000086017480068401C154908600020164954
:103CA000086040F224410D4800F0B6FF70B10B48A7
:103CB0000088C5B20948001D0088C5B20C480168DB
:103CC0000C48FFF75EFF00200949086070BD000046
:103CD0000038014000080140000C0140004800404D
:103CE00000440040000800406C010020C62B00206A
:103CF00060010020EA2A00206401002070B540F233
:103D00002551174800F088FFA0B1154800F004FFC6
:103D1000C4B214480068632804D2134811490968E2
:103D2000445402E000200F4908600E480068401C1F
:103D30000C49086040F22441094800F06DFF68B169
:103D400007480088C5B20648001D0088C5B206496C
:103D500006A001F0C5FE00200249086070BD000009
:103D60000038014068010020622B0020257300000C
:103D70000948804709480047FEE7FEE7FEE7FEE7FF
:103D8000FEE7FEE7FEE7FEE7FEE7FEE7044805493B
:103D9000054A064B704700005B050008310100082A
:103DA000902C002090320020902E0020902E002099
:103DB00031490143314A1160704770B50021002339
:103DC0000F22C47804B32D4C246804F4E064C4F5D5
:103DD000E064210AC1F10403CA40447804FA03F103
:103DE0008478144021430901254C0678A1550478B4
:103DF00004F01F050124AC4005786D11AD0005F1FC
:103E0000E025C5F8004109E0047804F01F0501240D
:103E1000AC401C4D0678761145F8264070BD1A4A14
:103E20000A400243154B1B1F1A60704739B1134AF1
:103E3000121D12680243114B1B1D1A6006E00F4A47
:103E4000121D126882430D4B1B1D1A607047042817
:103E500008D14FF0E021096941F004014FF0E02260
:103E6000116107E04FF0E021096921F004014FF0F2
:103E7000E0221161704700000000FA050CED00E03F
:103E800000E400E080E100E080FFFF1F10B5044681
:103E9000CC48844208D10121042000F02DFB0021F0
:103EA000042000F029FB46E0C748844208D10121E4
:103EB000082000F021FB0021082000F01DFB3AE063
:103EC000C248844208D10121102000F015FB0021D6
:103ED000102000F011FB2EE0BD48844208D10121E2
:103EE000202000F009FB0021202000F005FB22E04B
:103EF000B848844208D10121402000F0FDFA002199
:103F0000402000F0F9FA16E0B348844208D10121BC
:103F1000802000F0F1FA0021802000F0EDFA0AE0A4
:103F2000AE48844207D10121801500F0E5FA002156
:103F3000A01500F0E1FA10BD10B50121084600F00F
:103F4000DBFA0021012000F0D7FA10BD2DE9F04185
:103F5000024600250026002000230024002791F8B7
:103F600003C00CF00F0591F803C00CF0100CBCF16D
:103F7000000F03D091F802C04CEA050591F800C08B
:103F8000BCF1000F31D0146800202BE04FF0010C81
:103F90000CFA00F3B1F800C00CEA03069E4220D1EF
:103FA00083004FF00F0C0CFA03F7BC4305FA03FC37
:103FB0004CEA040491F803C0BCF1280F06D14FF07D
:103FC000010C0CFA00FCC2F814C00AE091F803C01E
:103FD000BCF1480F05D14FF0010C0CFA00FCC2F8FF
:103FE00010C0401C0828D1D31460B1F800C0BCF147
:103FF000FF0F34DD546800202EE000F1080C4FF074
:10400000010808FA0CF3B1F800C00CEA03069E425E
:1040100021D183004FF00F0C0CFA03F7BC4305FAD3
:1040200003FC4CEA040491F803C0BCF1280F05D14D
:1040300000F1080C08FA0CF8C2F8148091F803C0DB
:10404000BCF1480F07D100F1080C4FF0010808FA45
:104050000CF8C2F81080401C0828CED35460BDE88C
:10406000F0814FF6FF710180022181700421C1703F
:1040700070470246002093680B400BB1012000E01E
:10408000002070470146886880B2704702460020D1
:10409000D3680B400BB1012000E0002070470146BF
:1040A000C86880B2704701617047416170470AB1CA
:1040B000016100E041617047C16070474FF4803298
:1040C0000A43826181618261826982697047024626
:1040D0000020434B18684FF68073184040EA0210E6
:1040E00008433F4B186070473E49C8617047F0B5C0
:1040F0000A46002300240021002500F00046B6F106
:10410000004F02D1364EF16901E0354E7168C0F3BF
:10411000034583B200F44016B6F5401F08D121F0E4
:1041200070612F4E766826F070662D4F7E6012E02B
:1041300000F48016B6F5801F06D1032606FA05F4B2
:10414000A14341F0706106E0460D360103FA06F620
:10415000B14341F0706122B1460D360103FA06F613
:10416000314300F00046B6F1004F02D11C4EF16120
:1041700001E01B4E7160F0BD30B500228B071C0FB3
:104180000F2303FA04F2164B08338C1053F8243033
:104190009343134C08348D1044F8253023468C107B
:1041A00053F824308C07240F00FA04F423430C4CFA
:1041B00008348D1044F8253030BD0A49DC310860E0
:1041C0007047000000080140000C01400010014051
:1041D0000014014000180140001C01400020014073
:1041E0000000014000002042DF48006840F001006C
:1041F000DD49086008464068DC490840DA49486003
:1042000008460068DA490840D7490860084600684F
:1042100020F4802008600846406820F4FE004860D2
:104220004FF41F0088607047CF49096821F480313E
:10423000CD4A11601146096821F480211160B0F562
:10424000803F03D0B0F5802F0ED106E0C649096843
:1042500041F48031C44A116007E0C349096841F460
:10426000A021C14A116000E000BF00BF704710B537
:1042700001460022002300204A11012A02D1BA4C33
:10428000236806E0022A02D1B74C236A01E0B64C4B
:10429000636A01F01F02012494401C400CB101200C
:1042A00000E0002010BD38B500200090002400255B
:1042B00000BF3120FFF7DBFF05460098401C00904F
:1042C0000098B0F5A06F01D0002DF2D03120FFF79B
:1042D000CEFF08B1012400E00024204638BD01468D
:1042E0000020A14A106820F0F80040EAC1001060E8
:1042F0007047A04908607047024600209A4B5868F2
:1043000020F47C1042EA01031843974B5860704731
:1043100098490866704701460020934A506820F08B
:1043200003000843506070478F48406800F00C005D
:104330007047014600208C4A506820F0F000084386
:104340005060704701460020874A506820F4E060C2
:1043500008435060704701460020834A506820F4AB
:10436000605040EAC1005060704729B17E4A527ADD
:1043700002437D4B5A7204E07B4A527A82437A4B65
:104380005A7270477B49D831086070470146002057
:10439000754A506820F4404008435060704700213F
:1043A000714A20321170704A82F82010012802D020
:1043B00004280AD104E001216B4A2032117005E083
:1043C0000521694A2032117000E000BF00BF70472C
:1043D0006949086070476449096A0143624A116289
:1043E0007047654944390860704730B500210022A4
:1043F000002400235C4D6D6805F00C0121B10429F7
:1044000005D0082923D105E05C4D056022E05B4D15
:1044100005601FE0544D6D6805F47012524D6D68D3
:1044200005F48034022505EB92421CB9544D5543E6
:1044300005600BE04C4D6D6805F400351DB1504D25
:104440005543056002E04D4D5543056002E04B4D7C
:10445000056000BF00BF444D6D6805F0F00109091B
:10446000484D6B5C0568DD4045603F4D6D6805F467
:10447000E061090A434D6B5C4568DD4085603A4D5B
:104480006D6805F46051C90A3E4D6B5C4568DD40BE
:10449000C560354D6D6805F44041890B3A4D6B5C44
:1044A000C568B5FBF3F5056130BD29B12E4A5269E7
:1044B00002432D4B5A6104E02B4A526982432A4B36
:1044C0005A61704729B1284A92690243264B9A6182
:1044D00004E0254A92698243234B9A61704729B1CF
:1044E000214AD2690243204BDA6104E01E4AD269B4
:1044F00082431D4BDA61704729B11B4AD2680243DF
:10450000194BDA6004E0184AD2688243164BDA602D
:10451000704729B1144A12690243134B1A6104E02F
:10452000114A12698243104B1A617047124940398F
:10453000086070470F49C86470470B49C8717047DD
:104540000948406A40F08070074948627047014658
:104550000020054A92680A400AB1012000E00020CC
:104560007047014988727047001002400000FFF850
:10457000FFFFF6FE000042428004424200127A0031
:1045800000093D00740100208401002010B504469C
:10459000BE48844208D101218014FFF7ADFF0021FD
:1045A000A014FFF7A9FF16E0B948844208D1012101
:1045B0000014FFF7AEFF00212014FFF7AAFF0AE066
:1045C000B448844207D10121C013FFF7A2FF0021A4
:1045D000E013FFF79EFF10BD10B50022028802F421
:1045E00041520B884C8823438C882343CC88234337
:1045F0000C8923434C8923438C892343CC8923434F
:104600001A430280838B4FF2FF74234083830B8A0B
:10461000038210BD2DE9F04F85B005460C464FF0E2
:10462000000902274FF000084FF0010B0026B246A8
:10463000A88B4FF240010840A88302202884B5F8D7
:104640001C90A068022801D100BF38E0A08810B9F2
:104650004FF0010B01E04FF0020B8D48854200D175
:1046600000E000BF6846FFF7C0FEDDF800A0E0886C
:10467000B0F5007F0AD14FEA1A2000EB800040001D
:10468000A168B0FBF1F0401D86B20BE04FEA4B1081
:10469000BAFBF0F000EB80004000A168B0FBF1F045
:1046A000401D86B20A20B6FBF0F606F00108A6EB24
:1046B0000800C0F34F074FF6FF7000EA0828022FEA
:1046C00001DBFF2F02DD02274FF00008E08840EAFF
:1046D000080038432884A088A189084361880843DA
:1046E0002188084340F4006040EA0909A5F81C90BD
:1046F00005B0BDE8F08F0021018041808180C1803C
:10470000018141818181C18107210182704700219E
:10471000018041808180C1800221816000218181EE
:10472000704721B1028842F04002028004E0028812
:104730004FF6BF731A400280704721B1828B42F45A
:104740008062828304E0828B4FF6FF331A408283BB
:10475000704730B5002400230C110125A540ABB2F1
:104760001AB185881D43858002E085889D43858038
:1047700030BD1AB183880B43838002E083888B436A
:1047800083807047818170470146888970474FF662
:10479000FF62914204D0028842F48072028004E0F9
:1047A00002884FF6FF631A400280704721B1828869
:1047B00042F00402828004E082884FF6FB731A40C4
:1047C0008280704702884FF2FF731A40028002888D
:1047D0000A4302807047018841F48051018070478C
:1047E00021B1028842F40052028004E002884DF6B2
:1047F000FF731A400280704702460020012901D051
:10480000108B00E0908A70470146088A7047B1F526
:10481000804F04D1028842F48042028004E0028882
:104820004BF6FF731A40028070470246002013893E
:104830000B400BB1012000E000207047CA43028109
:104840007047F0B50246002000240023002501F047
:104850000F070126BE40B4B20B1101269E40B3B231
:10486000968806EA03051689264016B10DB1012087
:1048700000E00020F0BD10B5002201F00F0401237C
:10488000A3409AB2D343038110BD00000030014021
:1048900000380040003C004010B50446FB4884420C
:1048A00009D101218803FFF727FE00214FF4804042
:1048B000FFF722FE32E0F648844209D10121480484
:1048C000FFF727FE00214FF40030FFF722FE25E01E
:1048D000F048844209D101218804FFF71AFE002123
:1048E0004FF48020FFF715FE18E0EB48844209D111
:1048F0000121C804FFF70DFE00214FF40020FFF74F
:1049000008FE0BE0E548844208D101210805FFF7C5
:1049100000FE00214FF48010FFF7FBFD10BD2DE9D4
:10492000F04786B005460E460024A24600BFA146C9
:104930000027B08900B100BF2F462C8A4CF6FF70CB
:104940000440F08804432C82AC894EF6F3100440F6
:10495000B08831890843718908430443AC81AC8A2B
:104960004FF6FF400440B0890443AC8201A8FFF732
:104970003CFDC648874202D1DDF810A001E0DDF819
:104980000CA0A88900F4004040B10AEBCA0000EB7B
:104990000A1031684900B0FBF1F807E00AEBCA00E1
:1049A00000EB0A1031688900B0FBF1F86420B8FB15
:1049B000F0F004012009642101FB1089A88900F4AA
:1049C000004040B1322000EBC900B0FBF1F000F034
:1049D0000700044308E0322000EB09106421B0FB1B
:1049E000F1F000F00F0004432C8106B0BDE8F08721
:1049F0004FF41651016000218180C18001810C219A
:104A0000418100218181704710B502460020108A43
:104A10004FF2FF0318400B884C8823438C882343B4
:104A2000CC8823431843108210BD002101804180AF
:104A30008180C180704721B1828942F40052828115
:104A400004E082894DF6FF731A4082817047F0B509
:104A50000346002400260025002040F66A17B942CC
:104A600000D100BF1846C1F3421401F01F06012710
:104A700007FA06F5012C01D10C3004E0022C01D11B
:104A8000103000E014301AB107682F43076002E0CD
:104A90000768AF430760F0BD1AB1838A0B43838276
:104AA00002E0838A8B4383827047028A4FF6F07359
:104AB0001A400282028A0A430282704782894FF2B8
:104AC000FF731A40828182890A438281704721B133
:104AD000828942F00202828104E082894FF6FD73EE
:104AE0001A4082817047028A4FF6DF731A400282B1
:104AF000028A0A430282704721B1028A42F480424C
:104B0000028204E0028A4BF6FF731A400282704769
:104B1000C1F308028280704701468888C0F308000C
:104B20007047818941F0010181817047028BD2B2C7
:104B30000283028B42EA012202837047028B02F455
:104B40007F420283028B0A430283704721B1828A2B
:104B500042F02002828204E0828A4FF6DF731A401C
:104B60008282704721B1828A42F01002828204E080
:104B7000828A4FF6EF731A408282704721B1828A8F
:104B800042F00802828204E0828A4FF6F7731A40EC
:104B90008282704721B1828942F40042828103E01F
:104BA0008289C2F30E028281704721B1828A42F467
:104BB0000062828204E0828A4FF2FF731A4082828E
:104BC0007047828A4FF6FB731A408282828A0A43B8
:104BD0008282704721B1828A42F00202828204E01E
:104BE000828A4FF6FD731A40828270470246002087
:104BF000B1F5007F00D100BF13880B400BB101203D
:104C000000E00020704701F40072B2F5007F00D18F
:104C100000BFCA430280704770B5024600240023DB
:104C20000025002040F66A16B14200D100BFC1F352
:104C3000421501F01F03012606FA03F3012D02D1EC
:104C40009689334006E0022D02D1168A334001E0F6
:104C5000968A33400C12012606FA04F41688344072
:104C600013B10CB1012000E0002070BD10B500228E
:104C7000002340F66A14A14200D100BF0A120124A9
:104C80009440A3B2DC43048010BD00000038014012
:104C90000044004000480040004C004000500040EC
:104CA00010B50446FE48844208D10121C014FFF724
:104CB00023FC0021E014FFF71FFCC4E0B4F1804F97
:104CC00008D101210846FFF724FC00210120FFF74D
:104CD00020FCB8E0F348844208D101210220FFF70C
:104CE00018FC00210220FFF714FCACE0EE488442DF
:104CF00008D101210420FFF70CFC00210420FFF75C
:104D000008FCA0E0E948844208D101210820FFF70F
:104D100000FC00210820FFF7FCFB94E0E4488442FB
:104D200008D101211020FFF7F4FB00211020FFF72C
:104D3000F0FB88E0DF48844208D101212020FFF702
:104D4000E8FB00212020FFF7E4FB7CE0DA48844206
:104D500008D101214014FFF7CFFB00216014FFF7B9
:104D6000CBFB70E0D548844209D10121C804FFF78C
:104D7000C3FB00214FF40020FFF7BEFB63E0D048E7
:104D8000844209D101210805FFF7B6FB00214FF449
:104D90008010FFF7B1FB56E0CA48844209D10121D7
:104DA0004805FFF7A9FB00214FF40010FFF7A4FB13
:104DB00049E0C548844208D101214020FFF7A9FB02
:104DC00000214020FFF7A5FB3DE0C048844208D108
:104DD00001218020FFF79DFB00218020FFF799FB38
:104DE00031E0BB48844208D101218015FFF791FBD7
:104DF0000021A015FFF78DFB25E0B648844209D1BC
:104E000001210804FFF778FB00214FF48030FFF701
:104E100073FB18E0B048844209D101214804FFF730
:104E20006BFB00214FF40030FFF766FB0BE0AB4853
:104E3000844208D101218804FFF75EFB00214FF472
:104E40008020FFF759FB10BD00220288944B984246
:104E50000ED0994B98420BD0B0F1804F08D0914BB7
:104E6000984205D0904B984202D0904B984204D182
:104E70004FF68F731A404B881A438D4B984207D0D8
:104E80008C4B984204D04FF6FF431A40CB881A430C
:104E900002808B8883850B880385814B98420BD0D9
:104EA000854B984208D08B4B984205D08A4B98424C
:104EB00002D08A4B984201D10B7A03860123838268
:104EC000704770B5002400220023058C4FF6FE7653
:104ED00035400584028C8388048B4FF68F752C40F7
:104EE000B51E2C400D882C43751E2A400D892A437F
:104EF0004D882A436A4DA8420BD06F4DA84208D076
:104F0000744DA84205D0744DA84202D0734DA842FA
:104F100013D14FF6F7752A404D892A434FF6FB759A
:104F20002A408D882A434FF6FF652B404FF6FF55E8
:104F30002B408D892B43CD892B4383800483CD88DF
:104F40008586028470BD70B5002400220023058C84
:104F50004FF6EF7635400584028C8388048B48F643
:104F6000FF752C404FF6FF452C400D884FF6FF761D
:104F700006EA05252C434FF6DF752A400D8906EA1F
:104F800005152A434D8806EA05152A43444DA842D3
:104F900002D0494DA8421DD14FF67F752A404D8958
:104FA0004FF6FF7606EA05152A434FF6BF752A40ED
:104FB0008D8806EA05152A434FF6FF352B404FF240
:104FC000FF752B408D8906EA85052B43CD8906EABE
:104FD00085052B4383800483CD880587028470BDBB
:104FE00070B5002400220023058C4FF6FF66354083
:104FF0000584028C8388848B4FF68F752C404FF686
:10500000FC752C400D882C434FF6FF552A400D8926
:105010004FF6FF7606EA05252A434D8806EA052560
:105020002A431F4DA84202D0234DA8421DD14FF262
:10503000FF752A404D894FF6FF7606EA05252A437B
:105040004FF6FF352A408D8806EA05252A434EF69D
:10505000FF752B404DF6FF752B408D8906EA05152F
:105060002B43CD8906EA05152B4383808483CD88A5
:105070008587028470BD70B5002200230024058C52
:105080004EF6FF7635400584038C8488828B48F683
:10509000FF752A404FF6FF452A400D8820E00000AA
:1050A000002C01400004004000080040000C0040BB
:1050B000001000400014004000340140004C01404A
:1050C000005001400054014000180040001C004006
:1050D00000200040004001400044014000480140E1
:1050E0004FF6FF7606EA05252A434DF6FF752B405D
:1050F0000D8906EA05352B434D8806EA05352B4315
:10510000FA4DA84202D0FA4DA84208D14BF6FF75DD
:105110002C408D894FF6FF7606EA85152C43848056
:105120008283CD88A0F84050038470BD828B4FF2FB
:10513000FF331A408283828B4FF6FF7303EA012309
:105140001A4382837047F0B50C46154600220021B1
:105150000026078C4EF6FF7C07EA0C070784828B3B
:10516000018C4FF6FF7707EA043640F6FF473A40D6
:105170004FF6FF7707EA05273A434FF6FF7707EA2E
:1051800003373A43D94FB8420ED0D94FB8420BD06B
:10519000B0F1804F08D0D74FB84205D0D64FB842B3
:1051A00002D0D64FB84206D14DF6FF77394046F4CB
:1051B0008057394305E047F6FF57394044F480579C
:1051C000394382830184F0BD828B4FF6F3731A401A
:1051D0008283828B0A4382837047F0B50C46154662
:1051E000002200210026078C4FF6FF6C07EA0C070F
:1051F0000784828B018C4FF6FF7707EA04264FF66F
:105200000C773A404FF6FF7707EA03172F433A43EC
:10521000B64FB8420ED0B64FB8420BD0B0F1804F67
:1052200008D0B44FB84205D0B34FB84202D0B34F04
:10523000B84206D14FF6FF57394046F480773943DC
:1052400005E04FF2FF57394044F4807739438283B9
:105250000184F0BD028B4FF2FF331A400283028BB0
:105260004FF6FF7303EA01231A4302837047F0B538
:105270000C461546002200210026078C4FF6EF7CD5
:1052800007EA0C070784028B018C4FF6FF7707EAC9
:10529000041640F6FF473A404FF6FF7707EA033718
:1052A0003A434FF6FF7707EA05273A438F4FB84254
:1052B0000ED08F4FB8420BD0B0F1804F08D08D4F39
:1052C000B84205D08C4FB84202D08C4FB84206D1BC
:1052D0004FF6DF77394046F01007394305E04FF6C7
:1052E0005F77394044F01007394302830184F0BDF1
:1052F000028B4FF6F3731A400283028B0A43028338
:105300007047F0B50C46154600220021068C4FF67A
:10531000FE773E400684028B018C4FF60C763240BD
:105320007E1C06EA03162E433243704EB0420ED066
:105330006F4EB0420BD0B0F1804F08D06D4EB042EE
:1053400005D06D4EB04202D06C4EB04206D14FF641
:10535000FD76314044F00106314305E04FF6F57625
:10536000314044F00106314302830184F0BD70B541
:1053700005460C465D4885420ED05D4885420BD0FF
:10538000B5F1804F08D05B48854205D05A48854228
:1053900002D05A48854200D100E000BF208850B9B1
:1053A0002389A28861882846FFF7ABFFE188284659
:1053B000FFF79EFF25E0208804280AD12389A288D0
:1053C00061882846FFF753FFE1882846FFF742FF30
:1053D00017E0208808280AD12389A28861882846F6
:1053E000FFF7FBFEE1882846FFF7EEFE09E0238980
:1053F000A28861882846FFF7A6FEE1882846FFF7C5
:1054000095FE70BD2DE9F04105460C4600260127AA
:10541000608808B9022600E00026A088012801D192
:10542000022700E001272088A0B92389A28861888B
:105430002846FFF766FFE1882846FFF759FF2389D2
:105440003A4631462846FFF712FFE1882846FFF723
:1054500001FF13E02389A28861882846FFF707FF30
:10546000E1882846FFF7F6FE23893A46314628466A
:10547000FFF747FFE1882846FFF73AFFBDE8F081D4
:105480000A884B881A438B881A43CB881A430B89A6
:105490001A434B891A438B891A43A0F8442070475A
:1054A0004FF6FF71818000210180C180418001722F
:1054B00070470021018041808180C180018141814C
:1054C0008181C1817047002101804180012181805B
:1054D0000021C180018170470021018041808180CD
:1054E000C18001814181818170470000002C014011
:1054F000003401400004004000080040000C00405F
:1055000021B1028842F00102028004E002884FF6D5
:10551000FE731A400280704731B1B0F8442042F463
:105520000042A0F8442005E0B0F84420C2F30E0287
:10553000A0F8442070471AB183890B43838102E0AD
:1055400083898B43838170478182704741EA0203DC
:10555000A0F8483070471AB183890B43838102E079
:1055600083898B438381704701894FF6F87211401C
:10557000018170470A46002101894FF68F73194057
:1055800011430181704730B504460D462946204637
:10559000FFF7F0FF208940F00700208130BD2DE9A2
:1055A000F04104460D4616461F46602D06D13B4687
:1055B000012231462046FFF75AFE05E03B46012214
:1055C00031462046FFF79DFE29462046FFF7D2FFD1
:1055D000208940F007002081BDE8F08130B50C46FD
:1055E00000210189C9B24FF6FF7505EA032515436D
:1055F00025432943018130BD2DE9F04105460E4682
:1056000017469846002443463A4631462846FFF757
:10561000E5FF2C894FF6F870044044F007044FF67C
:105620008F70044044F070042C81BDE8F081F0B527
:1056300004460D4616461F463B463246294620463E
:10564000FFF7CCFF208940F480402081F0BD018528
:10565000828270470A46002101884FF68F731940F5
:10566000114301807047F0B50C4615461E460021D7
:10567000002200230189028B038C4FF6F877394012
:1056800021434FF6FC473A4040F201173A434FF6A8
:10569000DD773B404FF6FF7707EA06172F433B4382
:1056A000018102830384F0BD0A460021018B4FF67D
:1056B0008F7319401143018370470A460021018B03
:1056C00048F6FF7319404FF6FF7303EA02231943AC
:1056D000018370470A460021818B4FF68F73194072
:1056E0001143818370470A460021818B48F6FF737E
:1056F00019404FF6FF7303EA022319438183704771
:1057000021B1028842F08002028004E002884FF654
:105710007F731A400280704721B1828842F00402F0
:10572000828004E082884FF6FB731A4082807047C3
:1057300021B1828842F00802828004E082884FF61C
:10574000F7731A408280704721B1828842F00102CB
:10575000828004E082884FF6FE731A408280704790
:105760000A460021018B4FF6F7731940114301835C
:1057700070470A460021018B4FF2FF7319404FF624
:10578000FF7303EA02231943018370470A4600218D
:10579000818B4FF6F77319401143818370470A4696
:1057A0000021818B4FF2FF7319404FF6FF7303EA1C
:1057B00002231943818370470A460021018B4FF66B
:1057C000FB7319401143018370470A460021018B86
:1057D0004FF6FF3319404FF6FF7303EA02231943D4
:1057E000018370470A460021818B4FF6FB731940F5
:1057F0001143818370470A460021818B4FF6FF33A6
:1058000019404FF6FF7303EA02231943818370475F
:105810000A460021018B4FF67F7319401143018323
:1058200070470A460021018BC1F30E014FF6FF734A
:1058300003EA02231943018370470A460021818B42
:105840004FF67F7319401143818370470A46002148
:10585000818BC1F30E014FF6FF7303EA0223194354
:10586000818370470A460021018C4FF6FD73194071
:105870001143018470470A460021018C4FF6F773EB
:1058800019401143018470470A460021018C4FF6EC
:10589000DF7319404FF6FF7303EA021319430184C3
:1058A00070470A460021018C4FF67F7319404FF66E
:1058B000FF7303EA02131943018470470A4600216B
:1058C000018C4FF6FF5319404FF6FF7303EA022392
:1058D0001943018470470A460021018C4FF2FF737F
:1058E00019404FF6FF7303EA0223194301847047FE
:1058F0000A460021018C4DF6FF7319404FF6FF73E5
:1059000003EA023319430184704730B500230124B0
:105910008C40A3B2048C9C430484048C02FA01F5ED
:10592000ADB22C43048430BD30B5002304248C4038
:10593000A3B2048C9C430484048C02FA01F5ADB23A
:105940002C43048430BD70B5034600200024184663
:10595000183001258D40ACB21D8CA5431D8409B1C2
:10596000082909D100EB6100056825F07005056084
:105970000568154305600EE00D1FC5F34E0528446C
:10598000056825F4E045056005684FF6FF7606EAF0
:1059900002263543056070BD21B1028842F0020243
:1059A000028004E002884FF6FD731A4002807047BF
:1059B00021B1028842F00402028004E002884FF61E
:1059C000FB731A400280704721B1828842F0800246
:1059D000828004E082884FF67F731A40828070478D
:1059E00002884FF6F7731A40028002880A43028049
:1059F000704782884FF68F731A40828082880A43EC
:105A00008280704702894FF6F8731A40028102893A
:105A10000A430281704702894FF67F731A40028160
:105A200002890A43028170478184704781857047EB
:105A3000818670470187704781877047A0F84010C2
:105A4000704702884FF6FF431A40028002880A43DB
:105A5000028070470146888E70470146088F704764
:105A60000146888F70470146B1F8400070470146F3
:105A7000888C70470146088D704702460020138AC3
:105A80000B400BB1012000E000207047CA430282A6
:105A9000704730B50246002000230024158A05EA2D
:105AA0000103958905EA010413B10CB1012000E05E
:105AB000002030BDCA430282704770471CB50C46B7
:105AC000064B7B4469460090204600F0F8FA0446F5
:105AD0000020694600F006FB20461CBD1F060000A2
:105AE0000FB4044910B503AA029800F017FB10BCCC
:105AF0005DF814FB7001002070B50C460546012AC4
:105B000005D02878800600D5EA69002302E0012349
:105B100005E05B1C934202D2E05C0028F9D1A86941
:105B2000E618C01AA861286A18442862284600F0BE
:105B3000DFF904E0D5E9012114F8010B9047B442E4
:105B4000F8D3284600F0EAF970BD0000F0B40D4625
:105B50000188090502D5214C7C4402E01F4C7C449D
:105B60000E34002100F1240608E002F00F071209AC
:105B7000E75D42EA03721B097754491C52EA0307A6
:105B8000F3D102780023120704D5702D06D009B195
:105B9000022311342246F0BC00F0E3B90123103493
:105BA000F8E770B504460D462146106800F0D0F9BC
:105BB000024629462046BDE870400023C6E7D21DB4
:105BC00022F00703D3E90023C0E70368126843F01B
:105BD000200303600823C3610023B7E78E4D000054
:105BE0002DE9F05F894604464FF0000ADFF874B1F2
:105BF000FB44C0F820A02046E1688847002874D004
:105C0000252806D0D4E901219047206A401C206253
:105C1000F1E700265F462046E168884720280546D0
:105C200007DB312D05D2781910F8200C08B1064396
:105C3000F1E7B00701D526F00406C4F81CA0002740
:105C4000C4F818A02A2D09D0284601F0C3FB38B3A8
:105C500004EB8708303DC8F8185019E059F8041BC8
:105C6000204604EB87029161E1688847012F0546D1
:105C700018D1E069002820DA26F020061DE0D8F8C7
:105C8000180000EB800005EB40003038C8F8180021
:105C90002046E1688847054601F09CFB0028EED1CC
:105CA000012F0AD02E2D08D12046E16888477F1C9D
:105CB0000546022F46F02006C4DBA069002803DA5F
:105CC000404246F00106A061F00701D026F0100620
:105CD0006C2D0BD0682D09D04C2D39D06A2D35D0C4
:105CE000742D35D07A2D33D016E038E0E1682F4698
:105CF00020468847B842054609D16C2F26D04FF47C
:105D00008060E168064320468847054604E06C2F22
:105D10001AD04FF4807006430DB3A5F14100192845
:105D200002D8203546F400664A46294620462660B9
:105D30004E46FAF757FA80B101280BD0F61D26F02F
:105D4000070000F1080956E74020E4E78020D8E783
:105D50000020D6E706F104094DE7284652E7206AFD
:105D6000BDE8F09F1E4D000030B505460B462A46A3
:105D700013F8014B12F8010B08B1A042F8D01CB186
:105D8000002802D06D1CF1E7284630BD10B5431C39
:105D900002E010F8011B71B18107FAD14FF0013216
:105DA00002C88C1A8C4314EAC211F9D0C01A0A0630
:105DB00003D0C01E10BDC01A10BD0A0401D0801E41
:105DC00010BD0902FCD0401E10BD431A28BF9A42E4
:105DD00040F28A82032A1044114440F2268010F0D7
:105DE000030F1EBF11F8013D521E00F8013D10F0D7
:105DF000030F7FF4F6AF11F0030300F0CD82083AF1
:105E0000C0F00B8051F8043D083A51F804CD40F839
:105E1000043D40F804CDFFF7F3BF121D5CBF51F8FD
:105E2000043D40F8043DAFF30080D20724BF11F8D1
:105E3000013D11F801CD48BF11F8012C24BF00F835
:105E4000013D00F801CD48BF00F8012C70474FF02C
:105E500000020429C0F0128010F0030C00F0C88288
:105E6000CCF1040CBCF1020F18BF00F8012BA8BF45
:105E700020F8022BA1EB0C0100F0BABA5FEAC17C5A
:105E800024BF00F8012B00F8012B48BF00F8012BBC
:105E9000704710B5044610F0030F08BF11F0030F50
:105EA00040F015804FF0013E121FC0F20E8051F8F5
:105EB000043BA3EB0E0C2CEA030C1CEACE1C08BF1F
:105EC00040F8043BF0D0A1F1040102F10402521E9B
:105ED00008DB11F8013B002B00F8013BF7D111461C
:105EE000FFF7B5FF204610BD7047704770477047F9
:105EF00070B5044685690068C10601D5302600E00A
:105F00002026C00707D070BDD4E901213046904754
:105F1000206A401C20626D1EF6D570BD70B5044627
:105F200085690078C00707D170BDD4E90121202020
:105F30009047206A401C20626D1EF6D570BD09682E
:105F40004A0501D540B27047C905FCD500B270477B
:105F500009684A0501D5C0B27047C905FCD580B2B1
:105F600070472DE9F0470D4699469246044600F1E8
:105F700024080168880604D5E06921F01001216039
:105F800000E00120A84201DD471B00E00027A169D5
:105F90007A1902EB0900081AA0612078C00602D421
:105FA0002046FFF7A5FF002608E0D4E901211AF8F2
:105FB00006009047206A401C761C20624E45F4DBA8
:105FC0002078C0060AD52046FFF792FF06E0D4E904
:105FD000012130209047206A401C2062381EA7F122
:105FE0000107F4DC07E0D4E9012118F80500904727
:105FF000206A401C2062281EA5F10105F3DC204622
:10600000FFF78CFF2078000602D50220BDE8F0875C
:106010000120FBE72DE9F0410646002410687529B0
:10602000314616A510D0FFF78AFF002802DA404259
:1060300013A507E031688A0701D512A502E04907D8
:1060400004D511A5012401E0FFF782FF00210A22F7
:1060500006F1240709E0B0FBF2FCB0FBF2F302FB0F
:106060001C00303078541846491C0028F3D12346D0
:106070002A463046BDE8F041FFF773BF000000003C
:106080002D0000002B0000002000000011680268B5
:10609000006A530501D508700AE0D30501D50880D0
:1060A00006E0130603D5C217C1E9000200E008604C
:1060B0000120704701694A1C02610878704700B5E9
:1060C0008FB0CDE901310021059105497944CDE931
:1060D000031011466846FFF783FD0FB000BD0000B6
:1060E000E5FFFFFF0A6802F8010B0A60704710B570
:1060F000436913B1AFF3008001E0FFF7FDFC01201D
:1061000010BD127800F124010A7000224A700122A9
:10611000EDE711684FF0FF32E9E70000074B70B57B
:106120000D467B44FFF7CBFF0446284600F0EFFB0B
:1061300010B14FF0FF3070BD204670BDBDD7FFFFDE
:106140002DE9FF5F15468A460446DFF8AC80F84427
:106150000027D8E900103E46CDE9001010E03AF8DB
:1061600016106A4602A800F0D6FB411C07D0217821
:10617000890603D5E269391891420DD80744761C87
:106180002078800602D5E069B84205DDAE42E6DB44
:106190003AF816000028E2D1A069C01BA061204691
:1061A000FFF7A6FED8E90010CDE90010002017E0A7
:1061B0003AF818106A4602A800F0ADFBB0F1FF3FB4
:1061C00081460BD000250DF1080B05E0D4E9012133
:1061D0001BF8050090476D1C4D45F7D308F10100F1
:1061E000B0428046E4DB206A384420622046FFF754
:1061F00095FEBDE8FF9F0000D24700002DE9F04169
:106200008046D21D22F007020025D2E90002F529BE
:1062100015A614D0011E72F1000106DA0023D0EB9E
:10622000030063EB020211A608E0D8F800108B0708
:1062300001D50FA602E0490701D50EA6012511469A
:10624000002408F1240704E000F0F7F830323A5552
:10625000641C50EA0102F7D12B46324621464046E3
:10626000BDE8F041FFF77DBE000000002D000000FA
:106270002B0000002000000030B4002100F12404B5
:1062800008E002F00705D208303542EA4372DB0825
:106290006554491C52EA0305F3D10468002310A297
:1062A000250707D5A40600D421B1C46901230DA296
:1062B000641EC46130BCFFF754BE10B504462146CD
:1062C0001068FFF745FE02462046BDE81040002357
:1062D000D2E7D21D22F00701D1E90023CCE700006C
:1062E0000000000030000000032A40F2308010F06F
:1062F000030C00F0158011F8013BBCF1020F624461
:1063000098BF11F801CB00F8013B38BF11F8013BF1
:10631000A2F1040298BF00F801CB38BF00F8013B9E
:1063200011F0030300F01783083AC0F0088051F819
:10633000043B083A51F804CBA0E80810F5E7121D19
:106340005CBF51F8043B40F8043BAFF30080D20738
:1063500024BF11F8013B11F801CB48BF11F8012B04
:1063600024BF00F8013B00F801CB48BF00F8012B27
:106370007047431A28BF9A4240F2ED82104410F051
:10638000030F11441EBF11F8013D521E00F8013DDC
:1063900010F0030F7FF4F6AF103AC0F00A8010B58A
:1063A00031E91850103A20E91850BFF4F9AFBDE8B0
:1063B0001040530724BF31E9081020E9081044BFFA
:1063C00051F8043D40F8043D12F0030F08BF704738
:1063D000D20728BF31F8023D48BF11F8012C28BF71
:1063E00020F8023D48BF00F8012C70474FF0000232
:1063F00000B5134694469646203922BFA0E80C50BB
:10640000A0E80C50B1F12001BFF4F7AF090728BF95
:10641000A0E80C5048BF0CC05DF804EB890028BF11
:1064200040F8042B08BF704748BF20F8022B11F03A
:10643000804F18BF00F8012B704730B5B0F10A0249
:106440004FEA900E71F100034EEA817EB0EB0E0030
:1064500061EB91014FEA101E4EEA017E10EB0E0037
:1064600041EB11114FEA102E4EEA016E10EB0E00B7
:1064700041EB11214FEA104E4EEA014E10EB0E0097
:1064800041EB1141401841F100014FEAD00040EAD0
:1064900041704FEAD10110EB80054FEA810444EAD4
:1064A000907444EB01046D1944EB0404521BA341A6
:1064B0004FF0000348BF0A3200D530BD401C41F107
:1064C000000130BD70472DE9FF4F0C461E464FF0CE
:1064D000FF378BB0D2E90001DDF860800A908A4670
:1064E000C1F30A5505B93D46002108464FF00000AA
:1064F000BAF1000F00F4400005DA00EB80004FF421
:10650000400101EA50004FEA9059B9F1010F00DD56
:10651000B9460A9850EA4A000ED044F61050A5F247
:10652000FF3545432F14B8F1000F1ED07542291EC8
:106530001EDDC9F100021CE0B8F1010F4FF00000B0
:1065400001D0302103E0F24305E02154401CB04269
:10655000FBDB30460022002121540B99C1F8088052
:10656000C1E900200FB0BDE8F08FBD1B6D1CDEE758
:106570004A4600DA694206A800F090FA06AB93E8B2
:10658000070003AB83E8070050460A9900F046FB7A
:106590008DE80700A0F500501F3800900398002DEB
:1065A0000ADD42F21F014A460844002303A9039072
:1065B000684600F0AFFD09E0A0F500504A461F38DC
:1065C000002303A90390684600F0B9FD8DE8070099
:1065D0000004000C03D04FF0FF30410800E01046EB
:1065E000B8F1000F03D00022009215461EE0751E80
:1065F00005D4FFF722FF303262556D1EF9D5B34640
:106600000122084302D000227F1C04E020783028B9
:1066100001D100227F1E002A099784D01DE0112D90
:1066200007DAFFF70AFF303262556D1C50EA0102AB
:10663000F5D1084302D00098C8B10EE00021681ED1
:1066400005E0235C625C63542254401E491C814275
:10665000F7DBAB46A81B401E0990002004F80B0096
:106660000B98099AC0F80880C0E9002B7AE7112638
:106670004FF0000857E72DE9F04F88460446D21D39
:1066800022F0070191B0D1E90001CDE90A0100F043
:106690008DFE02460B98C00F01D02D2007E0206828
:1066A000810701D52B2002E0202101EAC000032A46
:1066B000099001D0072A05DB03464146204600F039
:1066C000ADF90BE12078800601D5E06900E00620F5
:1066D000B8F1650F814606D0B8F1660F18D0B8F151
:1066E000670F70D131E00020B9F1110F009001DB8C
:1066F000112301E009F101030AAA01A90CA8FFF77F
:10670000E2FEDDE90C70002609F10105834647E051
:1067100001204B4600904FF000470AAA01A90CA89F
:10672000FFF7D1FEDDE90DB00C995D46002610B9EA
:1067300009F101000D18B9EB050003D4C0F1FF36D3
:1067400009F10105A5EB09002BE0B9F1010F01DA10
:106750004FF001090020B9F1110F0090484601DD0A
:10676000112300E003460AAA01A90CA8FFF7ABFE1B
:10677000DDE90C704D4600268346207800070AD4D8
:10678000AB4500DA5D4601A8012D04DD411911F881
:10679000011C302907D04F4502DA17F1040F04DA43
:1067A000012082460FE06D1EEEE7002F02DCED1B9C
:1067B0003E4403E0781CA84200DD7D1CB81B00F1BC
:1067C000010A4FF000472078000703D4AA4501DBF7
:1067D0004FF0FF3A0021B7F1004F0DF143088DF85B
:1067E000431024D002202B23002F01DA7F422D23D7
:1067F0000A21021EA0F1010000DC5FB197FBF1FC51
:1068000097FBF1F201FB1C7C17460CF1300C08F8E9
:1068100001CDEEE7A8F1010003702188090501D53B
:10682000452100E06521A0F1010800F8011C09984C
:106830000FA9A1EB0807FF1D00B10120411901EBD1
:10684000EA70A1693844081A401EA0612078C00689
:1068500002D42046FFF74CFB099828B1D4E9012166
:106860009047206A401C20622078C00622D520462E
:10687000FFF73EFB1EE0002E04DBB34502DD01A85E
:10688000805D00E03020D4E901219047206A401C5F
:106890002062761CAAF101005FEA000A0AD100F02A
:1068A000B9F8C0680168405CD4E901219047206ACA
:1068B000401C2062281EA5F10105DCDC07E0D4E9BC
:1068C000012118F8010B9047206A401C2062381EF5
:1068D000A7F10107F3DC2046FFF720FB032011B0EE
:1068E00041E610B5436913B1AFF3008001E0FFF753
:1068F00027FC012010BD128800F1240182840022AF
:10690000C2840122EDE711684FF0FF32E9E7007B16
:1069100000F08000704770B516460C46054600F042
:1069200071F8036893F80101012806D0FF2C0FD8F5
:10693000185D68B101202C7070BDD3F80701324694
:10694000214603F2071303442846BDE87040184768
:106950004FF0FF3070BD10B5203AC0F00B80B1E8A9
:106960001850203AA0E81850B1E81850A0E8185084
:10697000BFF4F5AF5FEA027C24BFB1E81850A0E88D
:10698000185044BF18C918C0BDE810405FEA827CA7
:1069900024BF51F8043B40F8043B08BF7047D207BE
:1069A00028BF31F8023B48BF11F8012B28BF20F85F
:1069B000023B48BF00F8012B7047754600F0EAF82B
:1069C000AE4605006946534620F00700854618B0DC
:1069D00020B5FDF7DBF9BDE820404FF000064FF091
:1069E00000074FF000084FF0000B21F00701AC4604
:1069F000ACE8C009ACE8C009ACE8C009ACE8C00923
:106A00008D46704710B500F005F8001D10BD00BFA1
:106A1000010A0000004870474C2C00202DE9F0418D
:106A20001F46044603260168072A01F4006004DBC0
:106A300008B116A505E016A503E008B115A500E00C
:106A400015A521F010002060A069C01EA0610FB143
:106A5000401EA0612046FFF74BFA4FB1D4E9012157
:106A600038469047206A401C2062C01C206206E025
:106A7000206AFAE7D4E9012115F8010B9047761E48
:106A8000F8D22046FFF74AFABDE8F0814E414E00A9
:106A90006E616E00494E4600696E66002DE9F04752
:106AA000814616468AB0354878440DC88DE80D00F9
:106AB00032487844801C03AC0DC884E80D0041F6D0
:106AC0009B300844372190FBF1F290FBF1F5A5F1E2
:106AD000800501FB12041B3C02D56442012000E04A
:106AE0000020DFF898A080460027FA44AAF1BE0AE9
:106AF0000EE0E0070AD03246684607EB4701012363
:106B00000AEB810100F01BFB8DE8070064107F1C7D
:106B1000002CEED1194F7F44AE3F19E0E80715D0A5
:106B200007EB04100DF1180A90E80E008AE80E0039
:106B3000C068F04201D1981908903246012306A995
:106B400003A800F0FCFA03AB83E807006D10641C97
:106B5000002DE3D14FF0010332466946B8F1000F32
:106B600003A802D000F0D6FA01E000F0E8FAC9E983
:106B70000001C9F808200AB0BDE8F087FC3E00001B
:106B800010B50446AFF300802046BDE81040F9F789
:106B90008CBB0000004870472C2C00204FF0013CBB
:106BA00050F8042B51F8043B9A4221D1A2EB0C037C
:106BB000934313EACC1317D150F8042B51F8043B3C
:106BC0009A4215D1A2EB0C03934313EACC130BD1D9
:106BD00050F8042B51F8043B9A4209D1A2EB0C0364
:106BE000934313EACC13DBD04FF00000704700BF93
:106BF000D01A01BAB1FA81F101F0180122FA01F0BC
:106C0000CB40C1F12001DBB2C0B2C01A2CFA01F3B3
:106C1000D11A914311EAC311E6D170475FEA400CE3
:106C200008BF91F0000F4FEA8C234FEAC12243EADC
:106C300051514FEA1C5018BF00F5F0404FEA3000A8
:106C400018BF41F000415FEA6C5C00F02980BCF1A4
:106C5000FF3F08BF40F080407047130C06BF12048E
:106C60004FF0100C4FF0000C130E04BF12020CF189
:106C7000080C130F04BF12010CF1040C930F04BF96
:106C800092000CF1020CD30F04BF52000CF1010C66
:106C900011464FF00002A0F11F00A0EB0C0070475E
:106CA00011F0004F08BF704731F000413FF4D5AFFD
:106CB0000B0C06BF09044FF0100C4FF0000C0B0E2C
:106CC00004BF09020CF1080C0B0F04BF09010CF101
:106CD000040C8B0F04BF89000CF1020CCB0F04BF16
:106CE00049000CF1010CCCF12003A0EB0C0022FABE
:106CF00003F302FA0CF241EA030100F101007047CC
:106D000020F07F4C80EA030023F07F47ACEB0703C1
:106D100003F57C5300F0004003F1FF032DE98049A7
:106D20004FEA154B09B44FEA144325EA0B4E24EA07
:106D300003480FF2042606EB132749083E785FEA62
:106D4000320203FB0667C7F5000707FB06F64FEAAA
:106D500054374FEAD64606F1020607FB066CCCF123
:106D6000005C4FEA1C472CEA074C07FB06F40CFBBF
:106D700006F504EB15464FEA961634BF00204FF097
:106D800000404FEAD13706FB07FC4FEA1C4C0CFBD6
:106D90000BF7D21B03FB0CF761EB07010CFB0EF7A3
:106DA000B0EB074072EB17420CFB08F734BFA2EBC5
:106DB0000742B2EB074261EB17414FEA0C444FEA3E
:106DC000910706FB07FC4FEA1C4C0CFB0BF7B0EBE2
:106DD000C74072EB573203FB0CF734BFA2EBC7423C
:106DE000B2EBC74261EB57310CFB0EF7B0EBC700BB
:106DF00072EB57720CFB08F734BFA2EBC702B2EB81
:106E0000C70261EB5771039F4FEA816141EA92111A
:106E100004EBCC044FEAD1374FEA826206FB07FC51
:106E200042EA90124FEA80604FEA1C4C0CFB0BF7D1
:106E3000D21B03FB0CF761EB07010CFB0EF7B0EB69
:106E4000074072EB17420CFB08F734BFA2EB074276
:106E5000B2EB074261EB17414FEA8C554FEA9107BD
:106E600004EB9C2406FB07FC4FEA1C4C0CFB0BF7C5
:106E7000B0EBC74072EB573203FB0CF734BFA2EB09
:106E8000C742B2EBC74261EB57310CFB0EF7B0EBD8
:106E9000C70072EB57720CFB08F734BFA2EBC702B6
:106EA000B2EBC70261EB577115EB4C254FEA8161DC
:106EB00041EA92114FEA82624FEAD13742EA9012D8
:106EC00006FB07FC44F100044FEA80604FEA1C4CCB
:106ED0000CFB0BF7D21B03FB0CF761EB07010CFB60
:106EE0000EF7B0EB074072EB17420CFB08F734BF0C
:106EF000A2EB0742B2EB074261EB174115EB1C1501
:106F00004FEA813141EA92414FEA823242EA9042AD
:106F10004FEA80304FEA0C7644F1000448EA03431C
:106F20004EEA0B484FF0000EB2EB080C71EB030772
:106F300024BF624639464EEB0E0E4FF0000B001890
:106F4000524149414BEB0B0BB2EB080C71EB0307C1
:106F50007BF1000B24BF624639464EEB0E0E4FF01C
:106F6000000B0018524149414BEB0B0BB2EB080CE4
:106F700071EB03077BF1000B24BF624639464EEBF1
:106F80000E0E51EA020718BF46F0010616EB0E7608
:106F900055F1000254F1000103D5BDE88901BDE8B7
:106FA0000088BDE88901BDE80048B619524141EBAF
:106FB0000101A3F10103704780807F7E7D7C7B7A95
:106FC0007978777676757473727171706F6E6E6D95
:106FD0006C6C6B6A6A69686867666665646463633B
:106FE00062616160605F5F5E5E5D5D5C5C5B5B5AC1
:106FF0005A5959585857575656555555545453532E
:1070000052525251515050504F4F4F4E4E4D4D4D88
:107010004C4C4C4B4B4B4A4A4A49494948484847D3
:107020004747474646464545454444444443434311
:107030004342424242414141002B9C4630D47700BA
:107040002BD01CB54FEA370703B44FF010004FF0B8
:107050001001BAF1000F06D0BCF1000FDCBF40F008
:10706000080040F008014FF000000FBCBDE81040E0
:107070000BF1010BBBF1010F08BF5FEA170722BF3D
:1070800012F1010211F101014FF0004143F100033F
:1070900000F0004043EA00007047F9D35708D0E7FA
:1070A00046EA064613F1400F4FEA16461FDD13F17C
:1070B000200FDFBF16430A46002120335B42BED0BB
:1070C000C3F1200746EA064602FA07F74FEA1646DA
:1070D00046EA0706C3F1200722FA03F201FA07F78E
:1070E00021FA03F14FF0000342EA0702A7E746EA5C
:1070F000020646EA06464FEA164646EA0106BCBFC5
:1071000046EA0646360C4FF000034FF000024FF0FF
:10711000000194E72DE9804C9A46934670B491E8BB
:10712000380007C831EA400C48BF34EA430C03D5A5
:10713000FFF7E6FDFFF780FFF0BCBDE8008C2DE90E
:10714000804C9A46934670B491E8380007C810F016
:10715000804F08BF13F0804F03D100F005F8FFF710
:107160006BFFF0BCBDE8008C20F07F4780EA030095
:1071700023F07F4C07EB0C03A3F57C5300F0004099
:10718000A3F1FE0392F0000F00F0B38095F0000F22
:1071900000F077802DE901494FEA11404FEA14468B
:1071A00021EA004800FB06FC24EA064708FB06F635
:1071B00007FB08F800FB07F718EB06484CEB164CEA
:1071C0004FEA124B18EB07484FEA15464CEB1740B5
:1071D00022EA0B4E0BFB06FC25EA06470EFB06F6E1
:1071E00007FB0EFE0BFB07F71EEB064E4CEB164C97
:1071F0004FF000061EEB074E4CEB174B18EB0B083D
:1072000040F1000018EB0E0B58EB000840F10000B5
:107210008F1A4FF000013CBFC943661B14BFB5EB8A
:10722000040C00213CBFC943F61B4FEA17444EEA49
:107230008E0E27EA04454FEA1C4704FB07622CEA3E
:10724000074C05FB07F70CFB05F604FB0CFC16EBE3
:10725000074642EB174216EB0C4642EB1C421BEB77
:10726000060658EB0202414146EA9E0601D5BDE8FA
:107270000189B619524141EB0101A3F10103BDE8B7
:1072800001894FEA14454FEA114724EA054621EAED
:10729000074C05FB07F406FB07F70CFB06F105FBA3
:1072A0000CFC11EB074144EB17444FEA124711EB7A
:1072B0000C4144EB1C4422EA074C05FB07F206FB99
:1072C00007F70CFB06F605FB0CFC16EB074642EB3A
:1072D000174216EB0C4642EB1C456A1854F10001AC
:1072E00048BF7047B619524141EB0101A3F10103B8
:1072F000704795F0000F37D04FEA11424FEA14471C
:1073000021EA024624EA074C02FB07F106FB07F7D5
:107310000CFB06F402FB0CFC14EB074441EB174199
:107320004FEA154714EB0C4441EB1C4125EA074C8E
:1073300002FB07F506FB07F70CFB06F602FB0CFC4D
:1073400016EB074645EB174516EB0C4645EB1C4282
:10735000121951F1000148BF7047B619524141EB73
:107360000101A3F1010370474FEA14454FEA1147A9
:1073700024EA054621EA074C05FB07F106FB07F75F
:107380000CFB06F24FF0000605FB0CFC12EB07426B
:1073900041EB174112EB0C4251EB1C4148BF7047C7
:1073A000921841EB0101A3F101037047490050EA33
:1073B000C12018BF04204A0D18BF40F0010040F260
:1073C000FF72B2EB515F08BF40F00200012808BF16
:1073D0000520704730380A2801D20120704700206C
:1073E0007047000010B500290AD00878002807D09F
:1073F00005487844FFF7D2FB002801D0002010BDDB
:107400000248784410BD0000EE350000E63500006B
:1074100010B500290AD00878002807D0054878441C
:10742000FFF7BCFB002801D0002010BD02487844C3
:1074300010BD0000DE350000D6350000FFF71BB997
:107440000000000000000000002F00000000070006
:10745000070000147F147F1400242A7F2A12006280
:10746000640813230036495522500000050300002C
:1074700000001C224100000041221C000014083EB4
:1074800008140008083E0808000000A0600000087A
:1074900008080808000060600000002010080402CE
:1074A000003E5149453E0000427F4000004261518C
:1074B0004946002141454B31001814127F10002726
:1074C00045454539003C4A494930000171090503E9
:1074D00000364949493600064949291E000036361A
:1074E000000000005636000000081422410000147D
:1074F000141414140000412214080002015109065A
:1075000000324959513E007C1211127C007F4949DA
:107510004936003E41414122007F4141221C007F0B
:1075200049494941007F09090901003E4149497A19
:10753000007F0808087F0000417F41000020404193
:107540003F01007F08142241007F40404040007FFF
:10755000020C027F007F0408107F003E4141413E43
:10756000007F09090906003E4151215E007F09198B
:1075700029460046494949310001017F0101003F88
:107580004040403F001F2040201F003F4038403F08
:10759000006314081463000708700807006151496C
:1075A000454300007F41410000552A552A550000FF
:1075B00041417F000004020102040040404040407D
:1075C000000001020400002054545478007F484415
:1075D000443800384444442000384444487F00384C
:1075E0005454541800087E0901020018A4A4A47C75
:1075F000007F080404780000447D4000004080843F
:107600007D00007F102844000000417F4000007C86
:1076100004180478007C0804047800384444443892
:1076200000FC242424180018242418FC007C0804DE
:10763000040800485454542000043F444020003CB7
:107640004040207C001C2040201C003C4030403C3E
:10765000004428102844001CA0A0A07C00446454CE
:107660004C44141414141414000000000000000012
:107670000000000000000000000000F80000000012
:10768000000000333000000000100C06100C060053
:10769000000000000000000040C07840C0784000BA
:1076A000043F04043F040400007088FC083000001C
:1076B000001820FF211E0000F008F000E018000074
:1076C00000211C031E211E0000F00888700000002D
:1076D0001E2123241927211010160E00000000007F
:1076E0000000000000000000000000E0180402009C
:1076F000000000071820400000020418E00000000D
:107700000040201807000000404080F0804040000A
:107710000202010F01020200000000F00000000060
:107720000101011F01010100000000000000000034
:1077300080B07000000000000000000000000000A9
:107740000001010101010101000000000000000032
:1077500000303000000000000000000080601804CD
:10776000006018060100000000E010080810E000AA
:10777000000F102020100F00001010F80000000073
:107780000020203F202000000070080808887000BA
:10779000003028242221300000300888884830003A
:1077A0000018202020110E000000C02010F800005A
:1077B00000070424243F240000F8088888080800F3
:1077C0000019212020110E0000E010888818000008
:1077D000000F112020110E0000380808C8380800DA
:1077E0000000003F0000000000708808088870005A
:1077F000001C222121221C0000E010080810E000DB
:107800000000312222110F00000000C0C000000063
:107810000000003030000000000000800000000088
:107820000000806000000000000080402010080080
:107830000001020408102000404040404040400049
:107840000404040404040400000810204080000024
:107850000020100804020100007048080808F00029
:107860000000003036010000C030C828E810E000F9
:107870000718272423140B000000C038E000000084
:10788000203C23020227382008F8888888700000EE
:10789000203F202020110E00C030080808083800C2
:1078A000071820202010080008F808080810E00039
:1078B000203F202020100F0008F88888E8081000DA
:1078C000203F20202320180008F88888E8081000AE
:1078D000203F200003000000C030080808380000E6
:1078E00007182020221E020008F808000008F808E7
:1078F000203F210101213F20000808F8080800006E
:107900000020203F2020000000000808F8080800A0
:10791000C08080807F00000008F888C02818080018
:10792000203F20012638200008F808000000000051
:10793000203F20202020300008F8F800F8F8080048
:10794000203F003F003F200008F830C00008F80842
:10795000203F200007183F00E01008080810E00052
:107960000F10202020100F0008F808080808F00069
:10797000203F210101010000E01008080810E0008C
:107980000F18242438504F0008F888888888700021
:10799000203F2000030C30200070880808083800C1
:1079A0000038202121221C00180808F808081800B7
:1079B0000000203F2000000008F808000008F80838
:1079C000001F202020201F000878880000C83808E9
:1079D000000007380E010000F80800F80008F80061
:1079E000033C0700073C03000818688080681808FB
:1079F00020302C03032C30200838C800C838080079
:107A00000000203F2000000010080808C8380800C7
:107A10002038262120201800000000FE020202006B
:107A20000000007F40404000000C30C0000000001B
:107A3000000000010638C00000020202FE00000043
:107A4000004040407F0000000000040202020400E9
:107A50000000000000000000000000000000000026
:107A6000808080808080808000020204000000000E
:107A70000000000000000000000080808080000006
:107A80000019242222223F2008F8008080000000F4
:107A9000003F112020110E000000008080800000B7
:107AA000000E112020201100000000808088F800C6
:107AB000000E112020103F200000808080800000F8
:107AC000001F222222221300008080F0888888185C
:107AD0000020203F20200000000080808080800067
:107AE000006B94949493600008F8008080800000FC
:107AF000203F210000203F200080989800000000D7
:107B00000020203F20200000000000809898000006
:107B100000C08080807F000008F800008080800026
:107B2000203F24022D302000000808F8000000004B
:107B30000020203F20200000808080808080800006
:107B4000203F20003F20003F808000808080000098
:107B5000203F210000203F20000080808080000026
:107B6000001F202020201F00808000808000000057
:107B700080FFA12020110E00000000808080800086
:107B8000000E112020A0FF80808080008080800077
:107B900020203F21200001000000808080808000A4
:107BA0000033242424241900008080E08080000019
:107BB0000000001F20200000808000000080800066
:107BC000001F202020103F208080800000808080C7
:107BD00000010E3008060100808000800080808057
:107BE0000F300C030C300F0000808000808080007C
:107BF0000020312E0E3120008080800000808080A7
:107C000080818E7018060100008080808080800056
:107C10000021302C2221300000000000807C020274
:107C200000000000003F404000000000FF00000096
:107C300000000000FF0000000002027C8000000045
:107C40000040403F00000000000601010202040461
:107C500000000000000000000000F888888888FF0D
:107C600088888888F80000000000000000000000FC
:107C7000000000000000000000001F080808087F46
:107C8000888888889F80F0000000000000000000C5
:107C900000000000000000000000FE0282828282DC
:107CA000FA8282828282020000000000000000004E
:107CB000000000000000000080601F404040404085
:107CC0007F40404458404000000000000000000099
:107CD00000000000000000000000F888888888FF8D
:107CE00088888888F800000000000000000000007C
:107CF000000000000000000000001F080808087FC6
:107D0000888888889F80F000000000000000000044
:107D100000000000000000001060028C0044645469
:107D20004D46445464C404000000000000000000FC
:107D3000000000000000000004047E0180403E00BE
:107D400000FE00007E80E000000000000000000057
:107D50000000000000000000080808F808080810EB
:107D600010FF101010F000000000000000000000E4
:107D700000000000000000001030101F088848308C
:107D80000E014080403F00000000000000000000A5
:107D900000000000000000000014A4442434AD667C
:107DA00024940444A414000000000000000000001B
:107DB000000000000000000008090808090909FD8A
:107DC00009090B0808090800000000000000000075
:107DD000000000000000000000FC848484FC00100F
:107DE00010101010FF101000000000000000000034
:107DF0000000000000000000003F1010103F0000D5
:107E0000010640807F00000000000000000000002C
:107E1000000000000000000020102CE7242400F0E7
:107E20001010FF1010F00000000000000000000023
:107E300000000000000000000101017F2111000787
:107E40000202FF0202070000000000000000000024
:107E50000000000000000000060909E6F80C04021A
:107E600002020202041E00000000000000000000E8
:107E70000000000000000000000000071F3020404C
:107E800040404040201000000000000000000000C2
:107E900000000000000000000000000000000000E2
:107EA00000000000000000003F4000000000000053
:107EB00000003000400030004000000009000BC00E
:107EC0003D000BC03D00090018C024407FE0224067
:107ED00031800000180024C01B000D80324001805A
:107EE00003801C4027401C800740004010006000B9
:107EF00000000000000000000000000000001F80E3
:107F0000204040200000402020401F800000000052
:107F1000090006001F80060009000000040004009C
:107F20003F8004000400000000100060000000001A
:107F3000000000000400040004000400040000002D
:107F4000000000400000000000000000002001C010
:107F500006003800400000001F80204020402040E4
:107F60001F800000000010403FC0004000000000E3
:107F700018C02140224024401840000010802040BA
:107F8000244024401B80000002000D0011003FC06F
:107F9000014000003C802440244024402380000015
:107FA0001F80244024403440038000003000200023
:107FB00027C03800200000001B80244024402440BB
:107FC0001B8000001C0022C0224022401F800000B5
:107FD0000000000008400000000000000000000059
:107FE0000460000000000000000004000A0011000E
:107FF0002080404009000900090009000900000034
:1080000000004040208011000A00040018002000F9
:1080100023402400180000001F80204027402940F2
:108020001F400000004007C039000F0001C00040A1
:1080300020403FC0244024401B8000001F8020407F
:10804000204020403080000020403FC020402040A1
:108050001F80000020403FC024402E4030C0000060
:1080600020403FC024402E00300000000F00108050
:10807000204022403380020020403FC00400040022
:108080003FC02040204020403FC020402040000012
:108090000060202020203FC02000200020403FC062
:1080A00024400B0030C0204020403FC02040004012
:1080B000004000C03FC03C0003C03C003FC0000087
:1080C00020403FC00C4023003FC020001F802040C4
:1080D000204020401F80000020403FC0244024005A
:1080E000180000001F802140214020E01FA0000058
:1080F00020403FC02440260019C0004018C0244042
:108100002440224031800000300020403FC0204009
:108110003000000020003F80004000403F802000F1
:1081200020003E0001C0070038002000380007C0D2
:108130003C0007C038000000204039C0060039C0AC
:10814000204000002000384007C0384020000000D8
:10815000304021C02640384020C000000000000010
:108160007FE0402040200000000070000C000380F1
:10817000004000000000402040207FE000000000A0
:10818000000020004000200000000000001000104F
:10819000001000100010001000000000400000005F
:1081A00000000000000002800540054003C00040C0
:1081B00020003FC004400440038000000000038012
:1081C00004400440064000000000038004402440B6
:1081D0003FC0004000000380054005400340000010
:1081E000000004401FC0244024402000000002E0A2
:1081F000055005500650042020403FC004400400B4
:1082000003C000400000044027C000400000000000
:1082100000100010041027E00000000020403FC0C4
:108220000140070004C00440204020403FC00040FF
:108230000040000007C0040007C0040003C00000A5
:10824000044007C00440040003C000400000038055
:108250000440044003800000041007F00450044070
:1082600003800000000003800440045007F0001069
:10827000044007C002400400040000000000064063
:108280000540054004C00000000004001F800440B9
:1082900000400000040007800040044007C0004088
:1082A0000400070004C0018006000400060001C0AD
:1082B000070001C006000000044006C0010006C01F
:1082C000044000000410071004E0018006000400D0
:1082D0000000044005C0064004400000000000000B
:1082E00004007BE040200000000000000000FFF0E0
:1082F00000000000000040207BE0040000000000BF
:1083000040008000400020002000400000000000ED
:10831000000000000000000000000000000000005D
:1083200000001FCC000C000000000000000008004E
:10833000300060000800300060000000022003FCF4
:108340001E20022003FC1E200220000000000E1848
:1083500011043FFF10840C78000000000F0010840F
:108360000F3800C0077818840078000000780F8468
:1083700010C411240E9800E400840008080068006E
:10838000700000000000000000000000000000007D
:10839000000007E01818200440020000000040021E
:1083A0002004181807E0000000000000024002400E
:1083B00001800FF001800240024000000080008038
:1083C00000800FF800800080008000000001000D98
:1083D000000E00000000000000000000000000800F
:1083E0000080008000800080008000800000000C81
:1083F000000C00000000000000000000000000066B
:10840000001800600180060018002000000007F03E
:10841000080810041004080807F000000000080411
:1084200008041FFC000400040000000000000E0C03
:1084300010141024104411840E0C000000000C18BD
:1084400010041104110412880C700000000000E0F8
:108450000320042408241FFC0024000000001F98AF
:10846000108411041104108810700000000007F03F
:1084700008881104110418880070000000001C0016
:10848000100010FC13001C001000000000000E384B
:1084900011441084108411440E38000000000700BD
:1084A000088C10441044088807F000000000000009
:1084B0000000030C030C000000000000000000009E
:1084C0000001010600000000000000000000008024
:1084D00001400220041008081004000002200220BD
:1084E00002200220022002200220000000001004CE
:1084F00008080410022001400080000000000E0067
:108500001200100C106C10800F00000003E00C181B
:1085100013E4142417C4082807D000000004003C0A
:1085200003C41C40074000E4001C000410041FFCAE
:108530001104110411040E880070000003E00C18EF
:1085400010041004100410081C10000010041FFC7C
:10855000100410041004080807F0000010041FFCA9
:108560001104110417C410040818000010041FFCA3
:108570001104110017C010000800000003E00C18DF
:108580001004100410441C780040000010041FFC6C
:1085900010840080008010841FFC10040000100470
:1085A00010041FFC10041004000000000003000170
:1085B000100110011FFE10001000000010041FFC2D
:1085C000110403801464181C1004000010041FFC24
:1085D0001004000400040004000C000010041FFC40
:1085E0001F0000FC1F001FFC1004000010041FFCF3
:1085F0000C04030000E010181FFC100007F008082E
:10860000100410041004080807F0000010041FFCF8
:1086100010841080108010800F00000007F00818F0
:1086200010241024101C080A07F2000010041FFC7C
:108630001104110011C011300E0C000400000E1CBA
:1086400011041084108410441C380000180010001D
:1086500010041FFC100410001800000010001FF888
:1086600010040004000410041FF8100010001E0085
:1086700011E0001C007013801C0010001FC0103C93
:1086800000E01F0000E0103C1FC000001004180CA8
:10869000163401C001C01634180C100410001C0060
:1086A000130400FC13041C00100000000804101C3C
:1086B0001064108413041C04101800000000000053
:1086C00000007FFE40024002400200000000300037
:1086D0000C0003800060001C00030000000040024A
:1086E000400240027FFE0000000000000000000089
:1086F0002000400040004000200000000001000178
:108700000001000100010001000100010000400023
:108710004000200000000000000000000000009861
:10872000012401440144014400FC000410001FFC2A
:10873000008801040104008800700000000000703F
:10874000008801040104010400880000000000709A
:1087500000880104010411081FFC0004000000F857
:10876000014401440144014400C800000000010428
:1087700001040FFC1104110411001800000000D6C0
:1087800001290129012901C90106000010041FFC6B
:10879000008401000100010400FC00040000010449
:1087A000190419FC0004000400000000000000038C
:1087B00000010101190119FE0000000010041FFC56
:1087C0000024004001B4010C01040000000010046A
:1087D00010041FFC0004000400000000010401FC60
:1087E0000104010001FC0104010000FC010401FC82
:1087F000008401000100010400FC0004000000F8F6
:10880000010401040104010400F80000010101FF5A
:108810000085010401040088007000000000007061
:10882000008801040104010501FF000101040104A5
:1088300001FC00840104010001800000000000CC64
:1088400001240124012401240198000000000100FA
:10885000010007F80104010400000000010001F814
:10886000000400040004010801FC00040100018070
:108870000170000C001001600180010001F0010C8A
:10888000003001C00030010C01F0010000000104C3
:10889000018C00740170018C010400000101018150
:1088A0000171000E001801600180010000000184C8
:1088B000010C013401440184010C0000000000009F
:1088C0000000000001003EFC4002400200000000E9
:1088D00000000000FFFF0000000000000000400258
:1088E00040023EFC010000000000000000006000AB
:1088F00080008000400040002000200000000000B8
:108900000000000000000000000000000000000067
:108910000000000000000000000000000000000057
:108920000000000000000000000000000000000F38
:1089300080380FFE380F8038000000000000000073
:108940000000000000000000000001000006000020
:108950000C00003800003100000600000C00003858
:10896000000030000000000000000000618000678F
:10897000F807F980006180006180006180006180FB
:108980000067F807F9800061800000000000000027
:10899000000001C0E003E0F00630080418081FFFE3
:1089A000FE040E080787F00381E0000000000000CD
:1089B00001F000060C00040408060C7001F9C00068
:1089C0000E00003BE000EC18070808040C18000338
:1089D000E00000000001E00007F003F818041C08A4
:1089E00004170807E1D003C0E00023B0003C0800F2
:1089F000200800001000000000000001000031000D
:108A0000003200001C000000000000000000000018
:108A10000000000000000000000000000000000056
:108A20000000000000000000000000007F0001FFC7
:108A3000C00780F00C0018100004200002000000A5
:108A40000000002000021000040C00180780F00154
:108A5000FFC0007F000000000000000000000000D8
:108A600000000000000000004200006600006600F8
:108A7000003C0000180003FFC0001800003C00008C
:108A800066000066000042000000000008000008C8
:108A90000000080000080000080001FFC0000800F6
:108AA00000080000080000080000080000000000A6
:108AB000000100003100003200001C000000000036
:108AC00000000000000000000000000000000000A6
:108AD0000000000008000008000008000008000076
:108AE0000800000800000800000800000800000856
:108AF0000000000000000000000000003800003806
:108B0000000038000000000000000000000000002D
:108B1000000000000000000000000000000600004F
:108B20001C000070000180000E0000380000C00032
:108B30000700001C000030000000000000000000E2
:108B40007F8001FFE0038070060018040008040025
:108B50000806001803807001FFE0007F800000001D
:108B600000000000000001000801000801000803E7
:108B7000FFF807FFF80000080000080000080000E8
:108B80000000000000000001C03802C05804009836
:108B9000040118040218040418061C1803F818012C
:108BA000E0F800000000000000000001C0E003C089
:108BB000F004000804080804080806180803F4185C
:108BC00001E7F00001E000000000000000000000EC
:108BD0000300000D00001100006100008108030186
:108BE0000807FFF80FFFF800010800010800000067
:108BF0000000000000E007FCD00608080610080688
:108C00001008061008061838060FF00607C0000006
:108C100000000000000000003F8001FFE0038430FE
:108C2000020818041008041008041008071810039C
:108C30000FF00007C000000000000000000003C0AB
:108C4000000700000600000600F80607F8061800F6
:108C500006E0000700000600000000000000000120
:108C6000E1E003F7F0063410041808041808040CB7
:108C700008040C0806161803F3F001C1E000000018
:108C800000000000F80003FC30030638040208046A
:108C900002080402080404100308F001FFC0007F6A
:108CA00000000000000000000000000000000000C4
:108CB00000000000703800703800703800000000BC
:108CC00000000000000000000000000000000000A4
:108CD0000000000000000000301A00301C000000FE
:108CE0000000000000000000000000000000000084
:108CF0000000000800001400002200004100008075
:108D0000800100400200200400100800080000005C
:108D100000000000210000210000210000210000CF
:108D2000210000210000210000210000210000217D
:108D3000000000000000000000000800080400100F
:108D4000020020010040008080004100002200005D
:108D5000140000080000000000000003C00004C070
:108D600000040000080038080F3808083808100010
:108D70000C300007E00003C000000000000000000D
:108D80003F8000FFE0038070020F1006708804C06F
:108D900088048308047F8802C09003012000FE40FD
:108DA0000000080000180001F8003E0801C200079A
:108DB000020007E20000FE00001FC80001F80000EA
:108DC0003800000804000807FFF807FFF804080847
:108DD00004080804080804080806180803F4180121
:108DE000E7F00001E0000000000000003F8001FF0C
:108DF000E003807002001804000804000804000862
:108E00000400100600200780C000000004000807CE
:108E1000FFF807FFF8040008040008040008040035
:108E20001802001003807001FFE0007F8000000046
:108E300004000807FFF807FFF804080804080804FE
:108E40000808040808043E08040008060018010089
:108E50006000000004000807FFF807FFF804080896
:108E6000040800040800040800043E000600000690
:108E70000000018000000000000000003F8001FFB2
:108E8000E0038070060018040008040208040208C9
:108E90000203F00783F0000200000200040008074C
:108EA000FFF807FFF80408080008000008000008A1
:108EB0000000080004080807FFF807FFF80400088E
:108EC0000000000000000400080400080400080777
:108ED000FFF807FFF8040008040008040008000079
:108EE0000000000000000000000600000700000174
:108EF00004000104000104000307FFFE07FFFC0457
:108F0000000004000004000004000807FFF807FF49
:108F1000F8040C08001800003E0004C7800503C8D0
:108F20000600F804003804001800000804000807D0
:108F3000FFF807FFF8040008000008000008000020
:108F40000800000800000800001800006000000091
:108F500004000807FFF807800807FC00007FC00036
:108F600003F80007C000780007800807FFF807FF34
:108F7000F804000804000807FFF807000803C00011
:108F800000E000003800001E000007000001C004DF
:108F900000F007FFF8040000000000007F8001FFE0
:108FA000E00380700600180400080400080600189A
:108FB00003003001FFE0007F80000000040008078C
:108FC000FFF807FFF8040408040400040400040484
:108FD00000040400060C0003F80001F0000000008B
:108FE000000000007F8001FFE0038070060088041D
:108FF00000880400C806003C03003E01FFE6007F35
:109000008400000004000807FFF807FFF8040808C0
:10901000040800040C00040F00040BC00610F00349
:10902000F03801E00800000800000001E0F803F05B
:1090300030063010041808041808040C08040C0842
:109040000206180207F00781E00000000180000618
:10905000000004000004000004000807FFF807FFF8
:10906000F80400080400000400000600000180006D
:1090700004000007FFE007FFF004001800000800EC
:10908000000800000800000800000804001007FFA6
:10909000E004000004000006000007E00007FE00F6
:1090A000041FE00001F80000380001E0043E000762
:1090B000C00006000004000004000007E00007FFF5
:1090C000C0041FF80007C007F80007FF80043FF83E
:1090D0000007C004F80007000004000000000004BE
:1090E000000806001807C07805F1C8003E00001F00
:1090F000800463E80780F8060018040008000000F8
:1091000004000006000007800007E008047C080057
:109110001FF80007F800180804E008070000060020
:10912000000400000000000100080600380400F8F8
:109130000403E8040F08047C0805F00807C00807CA
:1091400000180400600000000000000000000000A3
:10915000000000000000003FFFFE2000022000028F
:109160002000022000022000020000000000000099
:10917000000008000007000000C0000038000006E2
:10918000000001C000003000000E000001000000DF
:109190000000000000002000022000022000022049
:1091A00000022000023FFFFE00000000000000005F
:1091B00000000000000000000000000000080000A7
:1091C00010000030000020000030000010000008F7
:1091D000000000000000000000000100000100008D
:1091E0000100000100000100000100000100000179
:1091F000000001000001000001000001000000006B
:1092000000000000002000002000001000001000FE
:10921000000000000000000000000000000000004E
:109220000000000000F00019F8001B1800220800E0
:109230002608002408002410003FF8001FF8000052
:109240000800001800000004000007FFF80FFFF0FE
:10925000001818001008002008002008003018002E
:109260001FF0000FC00000000000000007C0001F3A
:10927000F0001830002008002008002008003C08FA
:10928000001C100000600000000000000000000052
:1092900007C0001FF0003818002008002008002038
:1092A0000804101007FFF80FFFF000001000000086
:1092B0000000000000000007C0001FF00012300096
:1092C0002218002208002208003208001E10000E9A
:1092D00020000000000000002000002008002008FE
:1092E00001FFF803FFF806200804200804200807FF
:1092F000200003000000000000000000000E000E2F
:109300006E001FF30031B10020B10020B100319197
:10931000001F13002E1E00200E003000000000046D
:10932000000807FFF80FFFF80010080020000020D9
:1093300000002008003FF8001FF8000008000000AF
:10934000000000000000002008002008002008069F
:109350003FF8063FF8000008000008000008000081
:1093600000000000000000000000000003000003F7
:10937000002001002001002003063FFE063FFC0004
:10938000000000000000000000000004000807FFCB
:10939000F80FFFF8000188000300002FC00038F824
:1093A0000020380020080000080000000000000035
:1093B000000004000804000804000807FFF80FFF7D
:1093C000F80000080000080000080000000000008D
:1093D000002008003FF8003FF800100800200000BF
:1093E0003FF8003FF8001008002000003FF8003F61
:1093F000F8000008000000002008003FF8003FF8D7
:10940000001008001000002000002008003FF800B5
:109410001FF80000080000000000000007C0000F57
:10942000F000183000300800200800200800300844
:10943000001830000FF00007C0000000000000001E
:109440002001003FFF003FFF001011002009002015
:1094500008002008003038001FF0000FC000000096
:109460000000000007C0001FF000381800200800AE
:109470002008002009001011001FFF003FFF00001E
:1094800001000000002008002008002008003FF82C
:10949000003FF80008080010080020080020000025
:1094A0003000003000000000000000000000000C50
:1094B00078001E18003308002308002108002188C6
:1094C0000021980030F0003860000000000000002B
:1094D000200000200000200000FFF003FFF8002023
:1094E00008002008002008000030000000000000F4
:1094F000000000002000003FF0007FF8000018008E
:109500000008000008002010003FF8007FF0000075
:1095100010000000000000002000003000003C00AF
:10952000003F800023F000007800007000238000DE
:109530003C00003000002000002000003C00003F04
:10954000E00023F80000E0002700003E00003FE0BC
:109550000021F80001E0003E0000200000000000B3
:109560002008002008003838003E680027800003EB
:10957000C8002CF80038380020180020080000002F
:10958000000000002000003003003C01003F830089
:1095900023EC000070002380003C0000200000202D
:1095A0000000000000000000000000380800203823
:1095B0000020F80023E8002F88003E08003808004B
:1095C00020180000700000000000000000000000F3
:1095D000000000000000000008000014001FF7FC5D
:1095E0003000062000020000000000000000000023
:1095F0000000000000000000000000000000FFFF6D
:10960000FF0000000000000000000000000000005B
:109610000000000000002000023000061FF7FC00E0
:10962000140000080000000000000000000000001E
:109630000000000000000018000060000040000072
:10964000400000200000100000080000040000049A
:1096500000000C00001000000000000000000000EE
:1096600000000000000000000000000000000000FA
:1096700000000000000000000000000000000000EA
:1096800000000000000000000000000000000000DA
:1096900000000000000000000000000000000000CA
:1096A000000001001A00130010000D000900000066
:1096B00000000000000000000000000001001A008F
:1096C000130001001A00100001001A000D00010033
:1096D0001A00090000000000000000000000000067
:1096E00000000000000000000000000002002C004C
:1096F00022001C00160010000100120000000000F3
:1097000000000000000001002C00220001002C00DD
:109710001C0001002C00160001002C0010000000AD
:109720000000000000000000000000000000000039
:109730000000000000000300460037002C0022005B
:109740001A000100160000000000000000000000E8
:10975000010046003700010046002C0002002300F3
:109760001100020023000D000000000000000000B6
:1097700000000000000000000000000000000000E9
:1097800004006400500040003000240001001A0072
:109790000000000000000000000001006400500014
:1097A00002003200200002003200180004001900FC
:1097B00009000000000000000000000000000000A0
:1097C00000000000000000000000050086006C00A2
:1097D00056003E002E0001001E00000000000000A8
:1097E00000000000010086006C00020043002B0016
:1097F000020021000F00020021000B000000000009
:109800000000000000000000020022001000020022
:1098100022000C000600AC0088006C004C003C00EC
:109820000100220000000000000000000000020013
:109830005600440004002B001B0004002B00130002
:1098400004002B000F0000000000000000000000DA
:109850000000000000000000000000000000070001
:10986000C4009C007C005800420002001600260044
:109870000000000000000000020062004E00040032
:1098800031001F00020020000E00040027000D0020
:1098900000000000000000000000000004002100A3
:1098A0000F00010028000E000800F200C2009A001C
:1098B0006E005600020018002A00000000000000A0
:1098C000000002007900610002003C002600040054
:1098D00028001200040028000E0000000000000014
:1098E00002003D00270002002900130002002900A9
:1098F0000F0009002401E800B600840064000200A3
:109900001A002E000000000000000000020092007B
:10991000740003003A002400040024001000040036
:1099200024000C0000000000000002003B002500A5
:10993000040025001100040025000D000A005A0152
:109940001201D8009A007A0002001C0032000000C8
:109950000000000000000200560044000400450022
:109960002B0006002B00130006002B000F00020046
:1099700057004500010046002C0002002C00140096
:1099800002002C0010000B0094014401FE00B40002
:109990008C0002001E0036000000000000000000E5
:1099A0000400650051000100500032000400320044
:1099B0001600030024000C0000000000000004005A
:1099C00051003300040033001700080025000D008B
:1099D0000C00D20172012201CE009E000200200084
:1099E0003A000000000000000000020074005C006B
:1099F00006003A00240004002E00140007002A008C
:109A00000E00020075005D0002003B00250006000C
:109A10002F00150004002B000F000D001402AC01F4
:109A20004E01F400B400020022003E0000000000DD
:109A300000000000040085006B0008003B002500CA
:109A400008002C0014000C0021000B000000000096
:109A5000000001003C00260004002D001500040059
:109A600022000C000E004502CD016D010501C5006C
:109A700003001A002E004200000000000000030056
:109A8000910073000400400028000B002400100027
:109A90000B0024000C00010092007400050041003E
:109AA0002900050025001100050025000D000F000C
:109AB0008F020B029F012701DF0003001A00300014
:109AC000460000000000000005006D005700050082
:109AD000410029000500360018000B0024000C008E
:109AE00001006E005800050042002A000700370000
:109AF0001900070025000D001000DD024D02C50110
:109B00004501FD0003001A0032004A000000000079
:109B1000000005007A006200070049002D000F00D8
:109B20002B00130003002D000F0001007B006300D9
:109B300003004A002E0002002C0014000D002E002D
:109B4000100011002F038702FB016F011B010300AE
:109B50001E0036004E0000000000000001008700DB
:109B60006B000A004A002E000100320016000200BD
:109B70002A000E00050088006C0001004B002F0039
:109B80000F003300170011002B000F001200850397
:109B9000D10233028D01390103001E00380052004A
:109BA0000000000000000500960078000900450054
:109BB0002B0011003200160002002A000E000100E6
:109BC00097007900040046002C00010033001700C4
:109BD00013002B000F001300DF031B037302BD01F2
:109BE000550103001E003A0056000000000000006E
:109BF00003008D007100030046002C0011002F00AF
:109C00001500090027000D0004008E0072000B00F3
:109C100047002D00040030001600100028000E0040
:109C200014003D045D039D02E50181010300220053
:109C30003E005A00000000000000030087006B0097
:109C40000300430029000F00360018000F002B000E
:109C50000F00050088006C000D0044002A0005007C
:109C6000370019000A002C00100015008404A4031A
:109C7000CA020002960104001C00320048005E0087
:109C800000000000040090007400110044002A004D
:109C900011003200160013002E0010000400910085
:109CA00075000000000000000600330017000600E9
:109CB0002F0011001600EA04EE030E033802BA0169
:109CC00004001A0032004A00620000000000020096
:109CD0008B006F0011004A002E00070036001800AC
:109CE000220025000D0007008C007000000000001D
:109CF00000001000370019000000000000001700ED
:109D0000540546045C036602D00104001E003600C0
:109D10004E00660000000000040097007900040077
:109D20004B002F000B003600180010002D000F0014
:109D3000050098007A000E004C0030000E0037003D
:109D400019000E002E0010001800C20596049203A0
:109D50009802020204001C00360050006A00000055
:109D60000000060093007500060049002D000B005E
:109D7000360018001E002E0010000400940076002B
:109D80000E004A002E0010003700190002002F00BC
:109D9000110019003406FC04E803CE021A02040084
:109DA00020003A0054006E0000000000080084000B
:109DB0006A0008004B002F0007003600180016004C
:109DC0002D000F00040085006B000D004C003000DA
:109DD0001600370019000D002E0010001A00AA0608
:109DE0005A052604F202540204001E003A005600EE
:109DF0007200000000000A008E00720013004A008A
:109E00002E001C003200160021002E00100002005F
:109E10008F00730004004B002F0006003300170072
:109E200004002F0011001B002407BC056804280350
:109E30007402040022003E005A0076000000000078
:109E4000080098007A00160049002D00080035002F
:109E500017000C002D000F00040099007B00030088
:109E60004A002E001A00360018001C002E001000B8
:109E70001C008107FB05A9046703950205001A0071
:109E800032004A0062007A0000000300930075006F
:109E9000030049002D000400360018000B002D00BF
:109EA0000F000A009400760017004A002E001F00E1
:109EB000370019001F002E0010001D0003085F0668
:109EC000F3048F03BD0205001E0036004E0066003D
:109ED0007E000000070092007400150049002D006C
:109EE00001003500170013002D000F00070093003C
:109EF000750007004A002E002500360018001A00E1
:109F00002E0010001E008908C7065D05D903E9026E
:109F100005001A0034004E006800820000000500B1
:109F20009100730013004B002F000F003600180043
:109F300017002D000F000A00920074000A004C0068
:109F4000300019003700190019002E0010001F0002
:109F500013093307AF050904190305001E00380073
:109F600052006C00860000000D009100730002009A
:109F70004A002E002A003600180017002D000F009E
:109F80000300920074001D004B002F0001003700F9
:109F900019001C002E0010002000A109A3070506CF
:109FA0005B044D03050022003C00560070008A004F
:109FB00000001100910073000A004A002E000A0000
:109FC0003600180013002D000F00000000000000F4
:109FD00017004B002F0023003700190023002E002C
:109FE00010002100330A17085F069304850305005B
:109FF0001E003A00560072008E0000001100910011
:10A0000073000E004A002E001D00360018000B00E1
:10A010002D000F0001009200740015004B002F006E
:10A020001300370019002E002E0010002200C90A6C
:10A030008F08BD06CF04C103050022003E005A0070
:10A040007600920000000D00910073000E004A009F
:10A050002E002C00360018003B002E0010000600D9
:10A060009200740017004B002F0007003700190002
:10A0700001002F00110023003C0B02091407060504
:10A08000DA0306001E0036004E0066007E009600D1
:10A090000C00970079000C004B002F0027003600C1
:10A0A000180016002D000F00070098007A001A0013
:10A0B0004C0030000E003700190029002E0010005F
:10A0C0002400DA0B82097A074A051E0406001800EC
:10A0D00032004C00660080009A000600970079006C
:10A0E00006004B002F002E003600180002002D0045
:10A0F0000F000E0098007A0022004C0030000A0089
:10A100003700190040002E00100025007C0C060AC4
:10A11000C8079205480406001C00360050006A007B
:10A1200084009E00110098007A001D004A002E0055
:10A1300031003600180018002D000F0004009900AF
:10A140007B000E004B002F000A00370019002E0084
:10A150002E0010002600220D8E0A3608DE05760439
:10A16000060020003A0054006E008800A20004009F
:10A1700098007A000D004A002E00300036001800CA
:10A180002A002D000F00120099007B0020004B00D8
:10A190002F000E003700190020002E0010002700AD
:10A1A000CC0DFC0AA8082E06C60406001A003600CC
:10A1B00052006E008A00A60014009300750028006B
:10A1C0004B002F002B00360018000A002D000F0056
:10A1D00004009400760007004C00300016003700A1
:10A1E000190043002E00100028007A0E8C0B1E0967
:10A1F0008206FC0406001E003A00560072008E0023
:10A20000AA0013009400760012004B002F002200D9
:10A210003600180014002D000F000600950077008E
:10A220001F004C0030002200370019003D002E00B6
:10A23000100001020408102040801D3A74E8CD8708
:10A2400013264C982D5AB475EAC98F03060C1830A2
:10A2500060C09D274E9C254A94356AD4B577EEC1DF
:10A260009F23468C050A142850A05DBA69D2B96FA5
:10A27000DEA15FBE61C2992F5EBC65CA890F1E3C1C
:10A2800078F0FDE7D3BB6BD6B17FFEE1DFA35BB611
:10A2900071E2D9AF4386112244880D1A3468D0BDCB
:10A2A00067CE811F3E7CF8EDC7933B76ECC59733B4
:10A2B00066CC85172E5CB86DDAA94F9E21428415B5
:10A2C0002A54A84D9A2952A455AA49923972E4D524
:10A2D000B773E6D1BF63C6913F7EFCE5D7B37BF68B
:10A2E000F1FFE3DBAB4B963162C495376EDCA557CB
:10A2F000AE4182193264C88D070E1C3870E0DDA7AC
:10A3000053A651A259B279F2F9EFC39B2B56AC4533
:10A310008A09122448903D7AF4F5F7F3FBEBCB8BD6
:10A320000B162C58B07DFAE9CF831B366CD8AD479D
:10A330008E010000011902321AC603DF33EE1B68DA
:10A34000C74B0464E00E348DEF811CC169F8C80866
:10A350004C71058A652FE1240F2135938EDAF012B6
:10A3600082451DB5C27D6A27F9B9C99A09784DE4BD
:10A3700072A606BF8B6266DD30FDE29825B31091B0
:10A38000228836D094CE8F96DBBDF1D2135C833811
:10A3900046401E42B6A3C3487E6E6B3A2854FA85E7
:10A3A000BA3DCA5E9B9F0A15792B4ED4E5AC73F378
:10A3B000A7570770C0F78C80630D674ADEED31C583
:10A3C000FE18E3A5997726B8B47C114492D92320CE
:10A3D000892E373FD15B95BCCFCD908797B2DCFCFF
:10A3E000BE61F256D3AB142A5D9E843C3953476D4F
:10A3F00041A21F2D43D8B77BA476C41749EC7F0C2C
:10A400006FF66CA13B52299D55AAFB6086B1BBCC6F
:10A410003E5ACB595FB09CA9A0510BF516EB7A754B
:10A420002CD74FAED5E9E6E7ADE874D6F4EAA850EC
:10A4300058AF57E59295EE6615FB432E3D764640A4
:10A440005E202D4A98B06456646A6882DACE8C4EDB
:10A4500008B73D5BCA25333A3AED8C7C05636978D1
:10A46000686B6D66A14C035BBF93A9B6C2E1782B04
:10A470008BCE4E2BEF7BCED69318639627F3A38813
:10A48000D7EA9E5EB86176AA4FBB9894FCB305628A
:10A490006099113C4F323DA31ABBCAB4DDE153EFC2
:10A4A0009CA4D4D4BCBED2ABF7F25DE60E6DDD3514
:10A4B000C84A08AC6250DB86A069A5E7E579873019
:10A4C000D375FB7E9FB4A998C0E2E4DA6F0075E80B
:10A4D0005760E315AD7D9E0267B6761191C96F1C7A
:10A4E000A535A115F58E0D6630E39991DA46A8DF02
:10A4F000C868E0EA6CB46EBEC393CD1BE8C9152BE7
:10A50000F5572AC3D477F225097B29AD9198D81F36
:10A51000B3B632306E56EF60DE7D2AADE2C1E08226
:10A520009C25FBD8EE28C0B40A066ABEF9A70443EE
:10A53000D18A8A20F27B591B78B9509C2645AB3CC6
:10A540001CDE5034FEB9DCF16F4D925E1A156C13AF
:10A55000695E71C1568CA37D3A9EE5EFDA67384695
:10A56000723DB781A70D623E8133C8B76210AC1F40
:10A57000F6EA3C987300A79871F8EE6B123FDA2563
:10A5800057D269B1784A79C475FB71E91E789F2268
:10A5900026E4E63BF35F31DAB0A414412D6F275176
:10A5A000317671DEC1FAF2A8D929A4F7B11EEE12F4
:10A5B00078993CC13B744FA1FC6280CD80A1F739F2
:10A5C000A338EB6A351ABBAEE268AA07AF23B572AF
:10A5D00058292FA37D864814E835230FFA67DDE656
:10A5E000191289E700033AF2DDBF6E54E608BC6A2F
:10A5F00060930F838B2265DF2765D5C7EDFEC97B8E
:10A60000ABA2C2753260BE073D7947F64537A8BC9C
:10A6100059F3BF19487B09910EF701EE2C4E8F3E7E
:10A62000E07E767244A334C2D993CCA925827166A8
:10A6300049B5705E5870FDE0CA73BB635905367149
:10A64000812C3A1087D8A9D3240104603CF14968D1
:10A65000EA08F9F577AE34199DE02BCADF13520FE3
:10A66000E419C482D3923C18FB5A2766F03DB23FEE
:10A670002E7B7312DD6F87A0B6CD6BCE5F9678B858
:10A680005B15F79C8CEEBF0B5EE35432A327226C64
:10A69000E87D9DA1A409762ED163CBC12303D16FA0
:10A6A000C3F2CBE12E0D20A07ED182A0F2D7F24BD7
:10A6B0004D2ABD2071417C45E472EBAF7CAAD7E8FE
:10A6C00085CD743256BA32DCFB59C02E567F7C13CE
:10A6D000B8E997D7160E3B9125F2CB86FE59BE5EA0
:10A6E0003B417C7164E9EB79164C566127F2C8DC7A
:10A6F0006521EFFE7433B71AC957D2DD71152E41AB
:10A700002D32EEB8F9E1663AD1DA6DA51A5FB8C01C
:10A7100034F523FEEEAFAC4F7B197A2B786CD75013
:10A7200080C9EB08993B651FC64C1F9C6A786B9DDE
:10A73000A4D87074025BF8A324C9CAE50690FE9BF6
:10A7400087D0AAD10C8B7F8EB6F9B1AEBE1C0A554C
:10A75000EFB8657C98CE6017A33D1BC4F7979ACAE3
:10A76000CF143D0A52741AF7421B3E6BFCB6C8B9AF
:10A77000EB37FBF2D2909AEDB08DC0F898F9CE5538
:10A78000FD8E41A57D17181E7AF0D60681DA1D913F
:10A790007F86CEF5751D293F9F8EE97D947B6B8C5E
:10A7A0001A0C098DF3C5E2C5DB2DD365DB781CB52A
:10A7B0007F0664F702CDC63973DB656DA05225268E
:10A7C000EE31A0D179560B7C1EB55419C2574166A3
:10A7D000BEDC461BD110590721F041CA716247DF28
:10A7E000F876D65E007A251702E43A790769874E33
:10A7F000F376464CDF594832466FC211D47EB523FA
:10A80000DD75EB0BE595937BD5287306C8641AF6C6
:10A81000B6DA7FD724BA6E6A2D33AF09079E9F310F
:10A8200044775C7BB1CCBBFEC84E8D95771A7F35E3
:10A83000A05DC7D41D18919CD096DAD104D85B2FA7
:10A84000B8922F8CC3C37DF2EE3F636C8CE6F21F8F
:10A85000CC0BB2F3D99CD5E70576DEB48888A23359
:10A860002E750DD751118BF7C5AB5FAD4189B24441
:10A870006F5F652948D6A9C55F072C9A4D6FEC28F4
:10A88000798F3F5750FDF07ED94D22E86A32A852A9
:10A890004C92436AAB19845D2D69F79FDF21E05D1F
:10A8A0004D465AA020FE2B965465BECD85343CCA39
:10A8B000A5DCCB975D540F54FDADA059E334C761BF
:10A8C0005FE734B1297D89F1A6E17602362052D7BF
:10A8D000AFC62BEEEB1B65B87F030508A3EE0A0C91
:10A8E0000E090B0D081010080A0C303132333435C4
:10A8F00036373839414243444546403058003031BC
:10A9000032333435363738396162636465664030D6
:10A9100078000400000800000000000000020001B0
:10A9200000001000000000000000000002400000D5
:10A93000000000A00000000005400000000000C86A
:10A94000000000000C4000000000409C00000000DF
:10A95000194000000020BCBE000000003440000090
:10A96000BFC91B8E00000004B5400000504BCFD083
:10A970006607E2CF010000006C4100003E8251AA50
:10A98000DFEEA73401000000D9420000DCB5A0E2F0
:10A990003A301F97FFFFFFFFB4450000FD25A0C818
:10A9A000E9A3C14FFFFFFFFFFF3F00000000008051
:10A9B00000000000FF3F00000000008000000000D9
:10A9C0000CAB000800000020880100006C010008AA
:10A9D000A8AB00088801002008310000C801000869
:10A9E0001C00000043000000F8FFFFFF0C00000007
:10A9F0000E0000000F0000002E00000010010000FB
:10AA000043000000F8FFFFFF00404040404040404E
:10AA10004040414141414140404040404040404031
:10AA200040404040404040404005020202020202D5
:10AA30000202020202020202022020202020202024
:10AA40002020200202020202020290909090909038
:10AA500010101010101010101010101010101010F6
:10AA6000101010100202020202028888888888886A
:10AA70000808080808080808080808080808080856
:10AA8000080808080202020240000000000000005E
:10AA900000000000000000000000000000000000B6
:10AAA00000000000000000000000000000000000A6
:10AAB0000000000000000000000000000000000096
:10AAC0000000000000000000000000000000000086
:10AAD0000000000000000000000000000000000076
:10AAE0000000000000000000000000000000000066
:10AAF0000000000000000000000000000000000056
:10AB00000000000000000000000000005184A24A84
:10AB10000400091C01020304060708091332A48279
:10AB2000089A390C5A430C1A50081A5F041A6F0419
:10AB30005A80145A92085AA6085ABC085AD4085A7D
:10AB4000EE084B0AA5085A28085A48085A6A085AB3
:10AB50008E085AB4085ADC084B06A6085A32085A1E
:10AB600060085A90085AC2085AF6084B2CA7085A8F
:10AB700064085A9E085ADA084B18A8085A58085A06
:10AB80009A08011C000F1E7F415D5D5D417F1F1112
:10AB900015111F17EF2D0102030404000900060719
:08ABA000080902040608000088
:0400000508000131BD
:00000001FF
